:020000040005F5
:10000000E0630020C1030500C9030500CB03050020
:10001000CD030500CF030500D1030500000000005B
:10002000000000000000000000000000D3030500F5
:10003000D503050000000000D7030500D903050023
:10004000E90D0500DB030500E1140500DB030500F5
:10005000DB030500DB0305004D0C0500D90E050090
:10006000B9140500DB030500DB030500DB03050015
:10007000DB030500DB030500DB030500DB030500F4
:10008000ED140500C90E0500DB030500DB030500C8
:10009000DB030500DB0305007B120500DB03050025
:1000A000DB030500DB030500CD140500DB030500C1
:1000B000DB030500DB03050000000000000000007A
:1000C000DB030500DB030500DB030500DB030500A4
:1000D000DB030500DB030500DB0305000000000077
:1000E0000000000000000000000000000000000010
:1000F0000000000000000000000000000000000000
:1001000000000000000000000000000000000000EF
:1001100000000000000000000000000000000000DF
:1001200000000000000000000000000000000000CF
:1001300000000000000000000000000000000000BF
:1001400000000000000000000000000000000000AF
:10015000000000000000000000000000000000009F
:10016000000000000000000000000000000000008F
:10017000000000000000000000000000000000007F
:10018000000000000000000000000000000000006F
:10019000000000000000000000000000000000005F
:1001A000000000000000000000000000000000004F
:1001B000000000000000000000000000000000003F
:1001C000000000000000000000000000000000002F
:1001D000000000000000000000000000000000001F
:1001E000000000000000000000000000000000000F
:1001F00000000000000000000000000000000000FF
:10020000DFF80CD000F010FA00480047B1460500B6
:10021000E063002030B450E8012F93B2C489234436
:100220008489A34228BF1B1B0489A34202BFBFF3DA
:100230002F8F002007E0C3EA020340E80134002CBE
:10024000E9D14FF001000A6030BC704750E8012F3F
:10025000C2EA024240E801210029F7D1704730B4D8
:1002600050E8022F1FFAA2F3C488A34202BFBFF3D3
:100270002F8F00200DE0C48923448489A34228BF26
:100280001B1BC2EA034340E80234002CE8D14FF0C4
:1002900001000A6030BC704750E8022FC2EA2242D7
:1002A00040E802210029F7D17047034653E8022FA6
:1002B000D988B2EB324F4FF0000017BF92B241EA3B
:1002C000014142EA014104E05A68B2EB324F08BFF3
:1002D000012043E80212002AE8D1704730B40446F6
:1002E00054E8000F0D4644E80053002BF8D1156088
:1002F00030BC704730B4044654E8000F40EA0105B2
:1003000044E80053002BF7D1156030BC704730B47F
:10031000044654E8000F00EA010544E80053002BAE
:10032000F7D1156030BC704730B4044654E8000F74
:1003300080EA010544E80053002BF7D1156030BC7A
:10034000704730B4044654E8000F00EB010544E860
:100350000053002BF7D1156030BC704730B4044611
:1003600054E8000FA0EB010544E80053002BF7D13F
:10037000156030BC704770B404464FF0000054E87C
:10038000006F0D68AE4207BF44E80023012044E837
:1003900000630E60002B1CBF0020F0E770BC7047AC
:1003A00030B4044654E8000F88422CBF451A054675
:1003B00044E80053002BF5D1156030BC70470000B5
:1003C0000648804706480047FEE7FEE7FEE7FEE7EF
:1003D000FEE7FEE7FEE7FEE7FEE7FEE79112050017
:1003E000010205002DE9F05F0546002092469B467C
:1003F00088460646814640241BE02846414647463B
:10040000224600F02FF853465A46C01A914110D3A5
:1004100011461846224600F016F82D1A67EB01081F
:100420004F4622460120002100F00DF817EB00098D
:100430004E41201EA4F10104DFDC484631462A4625
:100440004346BDE8F09F202A04DB203A00FA02F17F
:10045000002070479140C2F1200320FA03F31943B2
:1004600090407047202A04DB203A21FA02F0002154
:10047000704721FA02F3D040C2F1200291400843B4
:1004800019467047004870477C9A050040EA01030E
:100490009B0703D009E008C9121F08C0042AFAD23A
:1004A00003E011F8013B00F8013B521EF9D27047FE
:1004B000D2B201E000F8012B491EFBD270470022A6
:1004C000F6E710B513460A4604461946FFF7F0FF53
:1004D000204610BD30B505462A460B4612F8010BE2
:1004E00013F8014B08B1A042F8D01CB1002802D08B
:1004F0006D1CF1E7284630BDCAB2401E10F8011F3E
:100500008A4202D00029F9D100207047421C10F81D
:10051000011B0029FBD1801A7047034611F8012BFB
:1005200000F8012B002AF9D11846704770B50F4D1D
:1005300000B92868002412E00A4602E09E4203D077
:10054000521C1378002BF9D1DAB2224305D02BB11B
:1005500024B1002100F8011B04E00446401C067889
:10056000002EE9D12860204670BD0000382F002001
:1005700070B5064601F06AF9046805460A220021B2
:10058000304600F018F82C6070BD30B50B460146BF
:1005900000202022012409E021FA02F59D4205D322
:1005A00003FA02F5491B04FA02F52844151EA2F1CC
:1005B0000102F1DC30BD2DE9F04791460F4680463F
:1005C0000446002614F8015B2DB1FFF75BFF0068BD
:1005D000405DC007F6D12B2D02D02D2D18D0641E02
:1005E0004A463946204600F031F827B13968A14221
:1005F00001D1C7F8008071054FF002040BD54042CD
:10060000002803DD01F022F90460A007BDE8F087AF
:1006100046F48066E4E70028F8DA01F017F9046090
:100620006FF00040F2E70000064C074D06E0E0687E
:1006300040F0010394E8070098471034AC42F6D329
:10064000FFF7E2FD90A30500B0A305002DE9F05FE0
:1006500082460078002715468B460AF10104B94608
:10066000302801D09DB113E014F8010B0127782840
:1006700003D0582801D045B10AE00DB1102D07D1A3
:100680000027102514F8010B02E0082500E00A25D8
:100690000026B0460EE005FB080005FB06F1012729
:1006A00001EB10461FFA80F8B6F5803F00D3B9463B
:1006B00014F8010B294600F018F80028EBDABBF11A
:1006C000000F05D00FB1641E00E05446CBF8004087
:1006D000B9F1000F06D001F0B9F802210160C81E7F
:1006E000BDE8F09F48EA0640FAE73A2800D23038E1
:1006F00020F02002412A01D3A2F13700884201D321
:100700004FF0FF30704770B58C1810F8015B15F092
:10071000070301D110F8013B2A1106D110F8012B73
:1007200003E010F8016B01F8016B5B1EF9D12B0798
:1007300005D40023521E0DD401F8013BFAE710F84E
:10074000013BCB1A921C03E013F8015B01F8015B3B
:10075000521EF9D5A142D8D3002070BD2DE9F04F2B
:10076000ADF5017D0E460525002201AF02E0815C5A
:10077000B954521CB242FAD39DF80400262852D034
:10078000E4A101A8FFF7A6FE0446E01B301A06B25A
:10079000022E67DD681CC2B2DFA1204602F030FCE9
:1007A000A0B10322DEA1204602F02AFCD0B303222E
:1007B000DCA1204602F024FC002853D10222DAA159
:1007C000E01D02F01DFC00284CD10925D74FFE800A
:1007D000D7A12046FFF77EFE4FF0000A70B3F988DC
:1007E000601810F8052C3D2A22D010F8062C3D2A5E
:1007F00020D010F8070C3D281ED00B26891B204660
:1008000004F024F91FFA80F8F61E1FFA86F9F8881A
:100810000421A0EB0900204403F06CFC80B24FF0EF
:10082000060B1BE002E001AC0025CFE70225CDE777
:100830000726E3E70826E1E70926DFE74FF001098D
:10084000F9882046491E04F001F900F0FF08F988F4
:10085000491E605C04F801A04FF0030B804505D0F1
:1008600087F803A00DF5017DBDE8F08F04EB0508C6
:10087000B0A1404602F0D4FBB049B14A0323891A23
:10088000C90803EB014598B14046AEA102F0C8FB90
:10089000AE4E002844D04046ADA102F0C1FB002876
:1008A00062D04046ACA102F0BBFB002873D025E12A
:1008B00041AAAAA1204608F0C4FA2C2141A8FFF7BA
:1008C0001BFEF0B1A7A141A8FFF730FEC7F81CA09E
:1008D000A4A10020FFF72AFEFFF74AFE00F6FF70F2
:1008E0006FF30B00C11700EB115003133B61284657
:1008F0009DA1FA6905F0ADFD0120B8700120F870E6
:10090000B0E7BB884FF0FF32A0A1A44800F08AFFF7
:10091000A248FFF7FBFDC1B2A04800F01DFAEDE7C9
:1009200041AA9FA1204608F08CFA8EA141A8FFF7AA
:10093000FDFDFFF71DFE024656F822107AB1192080
:1009400091FBF0F35B1C97A1944800F06BFF934878
:10095000FFF7DCFDC1B2914800F0FEF982E73239C1
:100960000C2091FBF0F3EDE741AA92A1204608F09C
:1009700068FA7CA141A8FFF7D9FDFFF7F9FD07460A
:1009800078A10020FFF7D2FDFFF7F2FD0446012C0D
:1009900002DA012403E028E0052C00DD05242346CB
:1009A0003A4680A17D4800F03DFF7C48FFF7AEFD50
:1009B000C1B27A4800F0D0F9284622467EA105F05F
:1009C00041FD8049F8B2087038B1641E04EBC401DF
:1009D00001EB041146F8201044E7641E04EB4400C8
:1009E000322101EB800030603CE741AA76A120462D
:1009F00008F027FA2C2141A8FFF77EFD20B159A16C
:100A000041A8FFF793FD0AE02E2141A8FFF774FDEE
:100A100020B16EA141A8FFF789FD00E041A80028A0
:100A20006CD0FFF7A5FD804618F1030F1CD0B8F17C
:100A3000000F93DB66A12046FFF74CFD0646300011
:100A40005CD0F988301B081AA0EB0900A0EB0B0062
:100A50003862002852DB284642465EA105F0F2FCCF
:100A6000002061493A6A06E001207870FAE63318FE
:100A7000DB780B54401C9042F9D35C4805F02AF80F
:100A800002463878009028465949FB6905F0E9FC90
:100A9000564805F01FF800289ED1387800289BD1D1
:100AA000F969414598D101203870CDF800A0B88887
:100AB0004D4A414301F5A0214C483B6A05F03EF9FF
:100AC000C7F814A0FB6928461A465B1C49A105F02B
:100AD000C0FCFB695B1CFB61BA884EA12F4800F08B
:100AE000A1FE2E48FFF712FDC1B22C4800F034F9E8
:100AF00028462A4A4BA105F0A5FCB3E64FA127489A
:100B000000F090FE2548FFF701FDC1B2234800F038
:100B100023F9A7E6543D0000543D59534D260000EB
:100B2000543D2600543D2E002E4D00009C2C0020EC
:100B300026433D0026475645523D000040A405008F
:100B4000C0A3050026474D453D000000182F00209A
:100B500026534D453D00000026463D004756455270
:100B6000000000002C000000666C6173685F646F19
:100B7000776E5F6E3D2025642065617273655F61ED
:100B80006C6C5F783D20256400000000543D2426F5
:100B90005645523D25642C2564000000004100208C
:100BA000474D4500543D2426524D453D25642C2596
:100BB00064000000534D45006D6F745F762025641E
:100BC00020200000302F0020460000002E000000F2
:100BD00026423D0020646F776E5F7061636B5F6ECD
:100BE00020203D202564200000420020402F0020CE
:100BF00078A20500206E72665F6673746F7261671B
:100C0000655F77726974653D202564202C2020255E
:100C100064000000543D242646474E3D25642C25A3
:100C2000640000003220504F52545F7320656E64A0
:100C30005F646174613D202573200000543D2426CB
:100C4000554E4B4E504152413D3000002DE9F84386
:100C50000025002000904FF4807801240026234FC7
:100C6000404605F0F5F938B1D7F80403204018B133
:100C7000404605F0E3F92543640008F104081FFA33
:100C800088F8761C082EEBD34FF4BE74204605F08E
:100C9000DFF948B1204605F0D1F945F000456A4634
:100CA0000121002005F082F915F0FF0F16D0012672
:100CB00000242E420ED007EB8401D1F81005C0F3BA
:100CC0000420D1F81015C1F30141094A52F824203B
:100CD00002B190477600641C082CEAD3002D02DA9A
:100CE000684607F0ADF8BDE8F883000000600040FA
:100CF000A036002010B507F0F7FA00F00FF806480C
:100D000007F04DFA04480C3007F049FA0248BDE8F4
:100D10001040183007F043BA0043002000B50648E1
:100D200000F00CF804480C3000F008F802485DF8B8
:100D300004EB183000F002B80043002001787B2952
:100D400009D07B21017041788170002101724172CC
:100D500081728180C180704730B5C1B0002201AD81
:100D600003E0835CAB54521CD2B28A42F9D32623EF
:100D70000A46491CC8B2AB544922411CC9B22A5484
:100D80003D22481CC4B26A54164B1A7892B12E21E7
:100D9000601CC0B22955411CC9B22A545A78481C5B
:100DA000C0B26A549A78411CC9B22A54DA78481CF5
:100DB000C4B26A5400200B49143122460B5C641CF7
:100DC000E4B2AB54401CC0B20328F6D3214601A8BC
:100DD00003F03CFE611CC9B2285501A806F066FB71
:100DE00041B030BDB42C002070B54FF48076304651
:100DF00004F051FC114DB40560B1304604F052FCD2
:100E00000120C4F80803687920B9012068712968B5
:100E1000002088474FF48276304604F03CFC0028DE
:100E20000AD0304604F03EFC0220C4F808032968CA
:100E3000BDE870400120084770BD0000982B0020DD
:100E400030B5B1F5FA6F08DA11F5FA6F05DD00215A
:100E50004161C1618161002030BD8469C268C5699A
:100E60000369624303FB05228568436905FB01337F
:100E70001A44426142F2107392FBF3F243689342C8
:100E800001DA1A4603E00368934200DD1A46C461A2
:100E90008161104630BDD1E900231A448B681A44A1
:100EA00082608B680A6802EB43025242C2608A6821
:100EB0000261CA68026009694160704700214161AE
:100EC0008161C1617047000002490248091F096839
:100ED00000680847202C00202DE9FE434FF482755E
:100EE000284605F089FC4A4F0024D8B1284605F071
:100EF0008BFC97F82E0010B197F82F0090B18DF869
:100F00000040786801903889ADF80800F96841B36D
:100F1000388B788379603881FC6039686846884707
:100F200087F82F4097F82E00012678B34FF4807889
:100F3000404605F061FC48B3404605F065FC7A8BFD
:100F400097F82D108A420ED9A2EB010082B27A8363
:100F50003889A0EB02007A6802EB400005F03AFC09
:100F60000FE03C74D9E707D1F86828B187F82F6003
:100F70007C8305F02FFC04E08A4202D187F82F60C1
:100F80007C83284605F040FC224806604FF48875B3
:100F9000284605F031FC48B1284605F035FC3C7484
:100FA00002208DF800003968684688474FF48A753A
:100FB000284605F021FC28B1284605F025FC3C74A4
:100FC000BDE8FE837C691FE0B4FA84F04FF0004175
:100FD000C1408C434FF48C7101EB8005284605F02D
:100FE0000BFC88B1284605F00FFC8DF80060A5F5D4
:100FF0008C75E8088DF8040045F38000401C8DF8DE
:101000000500396868468847002CDDD1D8E7000024
:10101000143700200470004000F07CBAF8B5044694
:101020000D4616460B4B1B78002B01D100F072FACF
:1010300000230093684600F0CDFF32462946204643
:1010400000F00AF804469DF8000000F0E5FF204695
:10105000F8BD00008C3D002070B50E4614461849BE
:1010600000EB400001EBC00518356869002806D088
:10107000012811D002281BD00024204670BD28462C
:1010800000F07CFAA04201D20024F6E72246314665
:10109000284600F0A4FBF0E7284600F06FFAA042D3
:1010A00000D2044622463146284600F098FBE4E789
:1010B00022463146284600F064FB0446DDE7000086
:1010C0008C3D00200FB408B504A900916A4603992D
:1010D00000F003F801B05DF814FB2DE9F04198B081
:1010E00080460C46164603A8139040201490002713
:1010F0001597CDF85C80169714F8011B39B1252996
:1011000017D013A800F01EFB16980028F4DA1698E2
:1011100000280ADD159820B103A94046159AFFF76B
:101120007DFFDDE9151008441690169818B0BDE84B
:10113000F081002101202278232A1ED02B2A18D0EA
:101140002D2A0ED0302A10D000200028F3D1257887
:10115000A5F130020A2A14D3002322782E2A17D0B0
:1011600023E041F00101641CEFE741F00201641C3F
:10117000EBE741F00401641CE7E741F00801641C5F
:10118000E3E7641C00EB800005EB40003038DEE74D
:10119000641C2578A5F130020A2A06D2641C03EBF0
:1011A000830205EB4203303BF3E76C2D0DD0682D35
:1011B0000BD0702D4ED00BDC252D58D0582D2FD0B4
:1011C000632D0CD0642D56D112E0641C2578ECE719
:1011D000732D31D0752D17D0782D4CD120E030688B
:1011E000011D31600078C1B213A800F0ABFA42E0F3
:1011F0003268151D35601568CDE900010A222946BF
:1012000013A800F0C7F936E03268151D356015687F
:10121000CDE900010A22294613A800F027FA2AE0A6
:101220003268151D35601568CDE900011022294688
:1012300013A800F01BFA1EE03068011D316005683C
:1012400015F8011BB9B113A800F07CFA1698002814
:10125000F6DA10E03068011D316001680820CDE940
:1012600000070346102213A800F000FA03E025212E
:1012700013A800F067FA641C46E705F09FBC000065
:1012800002490148086070470090D003342F0020C5
:1012900070B503F075FE4FF0805528B1B5F8240302
:1012A0007849C0F30420086003F0BEFE10B177490E
:1012B0007548486703F016FF28B1D5F84402744911
:1012C000C0F34230086003F037FF20B17148016875
:1012D00021F08071016003F051FF002428B16E48B5
:1012E000046044606A48001F046003F071FF18B195
:1012F000674903206431086003F08CFF68B16749D7
:10130000052008606549012078310860634808308D
:10131000046062493F20091D086003F09DFFE8B3A7
:101320005F4800685F4908605D48001D0068091D4E
:1013300008605B4808300068091D086058480C3098
:101340000068091D0860564810300068091D0860D3
:10135000534814300068091D08605148183001686E
:101360005048203001604E481C3000684D492431FF
:1013700008604B4820300068091D08604848243048
:101380000068091D0860464828300068091D08608B
:1013900043482C300068091D086000E019E040480F
:1013A000303000683F49403108603D4834300068C3
:1013B000091D08603A4838300068091D086038483F
:1013C0003C300068091D0860354840300068091D40
:1013D000086003F0ABFD28B1D5F85802324900F09F
:1013E0004F00086003F0F6FD30B130480168C907CE
:1013F00002D06FF00101016003F038FE20B12C48EB
:10140000016841F48061016022487438016841F448
:1014100070010160BFF34F8FBFF36F8F03F044FE85
:101420004FF0102220B1D2F8080219491C3108608F
:10143000D2F80002002803DBD2F8040200281CDAEC
:10144000012006F059F81523C2F8003206F05AF8C8
:10145000C2F8043206F056F8002006F04DF8BFF34B
:101460004F8F0C48F0380168124A01F4E0611143D3
:101470000160BFF34F8F00BFFDE7BDE87040FFF78D
:10148000FFBE0000403501400DF0ADBA00C007407E
:101490003C050040FCED00E00C010040105600400F
:1014A0000404001020C50040E40E00400004004089
:1014B0003C1700400400FA0504220249024802F0E9
:1014C00025BF0000FC3600200080004006220249B3
:1014D000024802F01BBF00000837002000A00140B6
:1014E0000148006800470000A02B002038B5074CD9
:1014F0002068002800D00120002806D00448406859
:101500008047002020602068009038BD0001014025
:10151000B42B002010B5124C02202061606111A094
:10152000A06104F17800E0614FF4007020620021B6
:10153000A1626162E1620BA0A06404F51E70E06428
:1015400010202065A1656165E16509A1E01DFEF738
:10155000E4FF08A12046FEF7E0FF2020A07110BDA7
:101560008C3D00205465726D696E616C0000000056
:101570005254540053454747455200000169C26820
:10158000914204D88068801A0844401E7047881A27
:10159000401E70472DE9FC5F0646DDE90C480F460A
:1015A00092469946C7F1000B002F01DA584600E039
:1015B0003846012502E090FBFAF06D1C5045FADA3E
:1015C000A94500D94D462CB1002F02DB5FEA4870D7
:1015D00000D5641E5FEA887002D5B9F1000F0FD004
:1015E0005FEAC8700CD144B90AE0641E202130467D
:1015F00000F0A8F8F068002802DB0CB1A542F4D393
:10160000F068002830DB002F05DA5F462D213046D8
:1016100000F098F806E05FEA487003D52B213046C9
:1016200000F090F8F06800281EDB08F003000228A4
:101630000FD1B9F1000F0CD144B90AE0641E30217A
:10164000304600F07FF8F068002802DB0CB1A542BC
:10165000F4D3F068002807DBCDE900484B4652463A
:101660003946304600F002F8BDE8FC9F2DE9F84FFE
:101670008246DDE90A4B88461746994640460125D1
:10168000012602E0B0FBF7F0761CB842FAD2B14571
:1016900000D94E465FEACB7018D1BCB15FEA8B70BF
:1016A00002D5B9F1000F02D0202000900BE03020CD
:1016B000009008E0641E5046009900F043F8DAF804
:1016C0000C00002802DB0CB1A642F3D3DAF80C00C0
:1016D00000280CDABDE8F88FA9F1010906E0B8FB93
:1016E000F5F0B84202D2DFF8589004E07D43B9F13A
:1016F000010FF4D9F0E7B8FBF5F000FB158819F8F5
:101700000010504600F01EF8DAF80C00002803DB49
:10171000B5FBF7F5002DEED15FEACB70DAD04CB90E
:10172000D8E7641E2021504600F00CF8DAF80C00CF
:101730000028CFDB002CCDD0A642F2D3CAE70000B0
:101740008498050010B50446A0686368421C934263
:1017500005D323681954A260E068401CE060D4E916
:101760000102824209D121682069FFF757FCA16874
:10177000884203D04FF0FF30E06010BD0020A06031
:1017800010BD2DE9F0470546894617464FF0000881
:10179000EC682869A04202D9061B761E03E0A968FE
:1017A000201A0E1A761EA868001BB04200D8064602
:1017B000BE4200D33E466868324620444946FEF7A2
:1017C00065FEB044B144BF1B3444A868A04200D1B8
:1017D0000024EC60002FDCD14046BDE8F0872DE905
:1017E000F041044688461646E768A068C51BE168D4
:1017F0006068B542084407D932464146FEF746FEC6
:10180000B819E060BDE8F0812A464146FEF73EFE89
:10181000761B08EB050132466068FEF737FEE6608E
:10182000F0E700000FB4084B10B504A902AA039812
:1018300000F038F8044602A9002000F0D4F9204650
:1018400010BC5DF814FB0000E71B05000048704762
:101850003C2F002002E008C8121F08C1002AFAD15C
:1018600070477047002001E001C1121F002AFBD120
:10187000704700000121202807DA81400848014212
:1018800001D00120704700207047402806DA203838
:10189000814001D00120704700207047012070472F
:1018A000FC06FFBD2DE9FF4F8BB08846054600269C
:1018B00006E025280BD0DDE90D1290476D1C761C43
:1018C00028780028F5D10FB03046BDE8F08F00240D
:1018D000A146A2460122AE4900E0044315F8013FAB
:1018E000203B02FA03F00842F7D128782A2810D0CA
:1018F0006FF02F022878A0F13001092915D809EBE3
:10190000890102EB410144F0020400EB01096D1C66
:10191000F0E758F8041B5FEA010903D544F40054CA
:10192000C9F1000944F002046D1C28782E2817D153
:1019300015F8010F44F004042A280ED06FF02F028E
:101940002878A0F1300109290AD80AEB8A0102EBB4
:10195000410100EB010A6D1CF2E758F804AB6D1C65
:1019600028786C280FD006DC4C2817D068280DD0BA
:101970006A2814D104E0742810D07A280FD10DE021
:1019800044F400140AE044F4801401E044F44014E8
:101990006978814202D104F580146D1C6D1C287891
:1019A000692865D006DC00288DD0632827D06428FC
:1019B00006D15DE06E2808D073282AD0752877D02C
:1019C000DDE90D129047761CE0E0C4F302500228D6
:1019D00009D003280DD0D8F8001004280DD00E60CF
:1019E00008F10408D2E0D8F80010F217C1E900624B
:1019F000F6E7D8F800100E80F2E70E70F0E718F85E
:101A0000041B8DF8001000208DF80100EB4601202A
:101A100003E058F804BB4FF0FF3061074FF00007B8
:101A200001D40AE07F1C57450DDA8742FADB1BF828
:101A300007100029F6D106E07F1C8742FCDB1BF86B
:101A400007100029F8D1DDE90D23A9EB0700814635
:101A5000214600F0B1F83044C61904E0DDE90D126A
:101A60001BF8010B90477F1EF8D22146484688E0BC
:101A700058F8040BC4F302514FF00A0B032900D1AC
:101A800000B2042900D140B2002802DA40422D21E0
:101A900002E0210505D52B218DF82410012104E059
:101AA00006E0E10710D02021F6E708AF089113E027
:101AB00058F8040BC4F302514FF00A0B032900D16C
:101AC00080B2042900D1C0B20021EEE75946FEF7EA
:101AD0005CFD303107F8011D0028F7D1ADEB0700A0
:101AE00000F1200B600702D524F4803401E04FF0B0
:101AF000010ADA4502DDAAEB0B0000E00020824675
:101B000000EB0B0108980144A9EB01000A90E003E7
:101B100006D4DDE90D2321460A9800F04DF806446D
:101B20004FF0000908E009A911F80900DDE90D12DC
:101B3000904709F10109761C08998945F3DBE00318
:101B40000CD5DDE90D2321460A9800F035F806444E
:101B500004E0DDE90D1230209047761CBAF1000157
:101B6000AAF1010AF5DC05E0DDE90D1217F8010B19
:101B70009047761CBBF10001ABF1010BF4DC0A9835
:101B80002146DDE90D2300F005F806446D1C97E6BB
:101B9000092801002DE9F041044600251E4617469C
:101BA000880404D405E039462020B0476D1C641E2B
:101BB000F9D52846BDE8F0812DE9F041044600251D
:101BC0001E469046C80301D5302700E02027880430
:101BD00004D505E041463846B0476D1C641EF9D572
:101BE0002846BDE8F0810A68531C0B6010707047EE
:101BF000800701D0002070470120704740680068CE
:101C0000401E084201D1012070470020704700218A
:101C1000425C0AB101207047491C0629F8D3002014
:101C20007047C3688B4206D811440069491E81423F
:101C300001D8012070470020704770B504460D465A
:101C400004F22740FFF7E3FF012D06D0022D0CD050
:101C5000032D0FD0042D15D110E0A17929B194F8EE
:101C6000241011B908B1012070BDE17911B108B19A
:101C7000022070BD207A08B1032070BD607A08B1DF
:101C8000042070BD002070BD401C0521B0FBF1F2A6
:101C900001FB1200704790F82400012801D01F209A
:101CA0007047EE20704710B501220221002001F09C
:101CB0000DF808B1072810D107220221012001F0F8
:101CC00005F808B1072808D100210A22084600F0CB
:101CD000FDFF08B1072800D1002010BD00B5ABB052
:101CE000AC216846FEF7EBFB02208DF800000120D6
:101CF0008DF8020006218DF80310ADF84C00124952
:101D000014918DF87C004021229144F2506123917E
:101D10000E4929918DF879008DF87B008DF87D00B2
:101D20004FF448702490002025908DF87800694683
:101D3000074800F017FB08B100F0ACF80121044897
:101D400000F00DFB2BB000BDE62A00201575050044
:101D50006830002010B50321044800F087FB0028FC
:101D600003D0BDE8104000F095B810BD68300020E9
:101D700070B50024064D06E06868012110F83400B3
:101D800005F038F8641C28788442F5D3002070BD33
:101D9000C02B0020F8B505460C4617460A2F01D285
:101DA0000720F8BD05F026F918B905F0E9F8002874
:101DB000F7D1134E75603470B76010211148FEF7EB
:101DC0007EFB0021316171610F4E0DE005EBC40017
:101DD0003168009181788DF8011000780B4A6946CE
:101DE00005F05EF80028DCD1641EE4B2EED2BDE856
:101DF000F84005480021064A001D00F05DB80000CB
:101E0000C02B002044370020BC960500B9400500D7
:101E10000537050072B604F0B3FB04F0DDF90028C5
:101E2000FBD111481149401AC408012000EB0440BD
:101E30000FA104F003FB11480068C00700D000BEEA
:101E4000022000EB04400EA104F0F8FABFF34F8F1C
:101E50000A48E43801680E4A01F4E0611143016068
:101E6000BFF34F8F00BFFDE740A40500C0A30500EE
:101E7000466174616C206572726F7200F0ED00E073
:101E800053797374656D207265736574000000008A
:101E90000400FA050EB500210091019102906A46F6
:101EA00044F20100FFF7B6FF0EBD0000014801F04B
:101EB0008CBC0000002C002010B5002A0BD000685C
:101EC0004FF0FF348460C4604261012905D00021D5
:101ED0000161002010BD072010BD0121F8E70000BE
:101EE00038B512484168009108235822104900680B
:101EF00003F0E4F9002807D10E4A69460E4801F0C4
:101F000069FC04460CB1204638BD01210A4801F0A5
:101F1000D0FC0123094A1946074801F02EFC064966
:101F2000012008390870204638BD0000C49605001D
:101F3000643700202D830500002C0020FFFF7F0068
:101F4000F8B504460E46174600250095684600F091
:101F500041F8D4E90201C04370EA01000ED09DF8B7
:101F6000000000F059F88DB1A761206900B1266129
:101F70002146BDE8F840002006F030BF02F082F8AC
:101F800080196941C4E902010125E8E70020F8BD94
:101F900038B5044600200090684600F01BF8D4E9EC
:101FA0000201C04370EA01000FD04FF0FF31A16081
:101FB000E16001259DF8000000F02EF83DB12146BA
:101FC000BDE83840012006F009BF0025F2E70020F7
:101FD00038BD000030B5EFF3108372B60B4A946839
:101FE0000121002C04D00170002B00D162B630BD5D
:101FF000916007490D68074C254015600C604C68DE
:1020000054604A174A6000210170EDE7BC37002098
:1020100080E100E0FC06FFBD09498A68002A0ED075
:1020200000280CD1EFF3108072B60B68054A1360DC
:102030004B68536000228A60002800D162B6704766
:10204000BC37002000E100E038B505460C4620888A
:10205000001D904201D90C2038BD684679DF002868
:10206000FAD12188032068542088401C80B2208047
:10207000192129542088401C80B220804119BDF8C4
:10208000000006F027FF218808442080002038BD8A
:10209000400C01D0002070470120704730B550EA55
:1020A000010206D041B100280DD013DAC0F10003BF
:1020B00011E04FF0000030BD002801DDFA2030BDF6
:1020C00040F2EE2030BD002901DD002030BD4FF48C
:1020D000FA7030BD0346002901DA4A4200E00A46A0
:1020E000194C9A420ADB02EBD275C3EB032303EBD4
:1020F000650393FBF2F254F822200CE003EBD37556
:10210000C2EB022202EB650292FBF3F254F82220AA
:10211000A2F6C412524241F28833002803DB0029A0
:1021200008DC9A1A06E0002903DD42F21070821AD8
:1021300000E01A440A2092FBF0F04FF47A7190FB11
:10214000F1F201FB120030BD6492050010B50020D1
:102150000A49D1F810442146012206E0C9680B79EA
:10216000834201D1002202E009680029F6D1002A49
:1021700003D1401C0A28EEDB501E10BD6C39002034
:1021800070B504461546002D09D00020286044B1E2
:10219000206840B1A079800707D0072070BD0E20CD
:1021A00070BD0E2070BD0E2070BD084600F03CFAD8
:1021B000C0B2142804D02179814203D8042070BD14
:1021C000052070BDE288216800FB02102860002015
:1021D00070BD2DE9FC4104460F46154600202E88AF
:1021E0000021298094F82D10002906D03246294676
:1021F000384600F02DFA002876D1A17831B1324668
:1022000029463846FFF720FF00286DD1E17841B11B
:1022100094F9030033462A46394601F0E6FC0028CB
:1022200062D1616841B191F9000033462A463946CE
:1022300006F037FE002857D1218951B1CDE900566B
:102240003B460622022104F1080006F015FF002893
:102250004AD1218A51B1CDE900563B4607220321DC
:1022600004F1100006F008FF00283DD1218B51B188
:10227000CDE900563B461522142104F1180006F062
:10228000FBFE002830D1D4F820C0BCF1000F07D0ED
:1022900033462A463946604601F01DF9002823D10D
:1022A000D4F824C0BCF1000F07D033462A46394683
:1022B000604602F053FB002816D194F82C1039B177
:1022C00033462A463946204606F0B0FA00280BD19C
:1022D0002178002908D002B033462A4639462046E4
:1022E000BDE8F04102F0D0BDBDE8FC8118B5044660
:1022F0000020009013466A46204600F007F818B107
:10230000BDF80000204418BD002018BD70B500289D
:1023100002D00AB1002404E0002070BD045D2C440A
:10232000A4B2651C8D4206D21688A642F6D80619BC
:1023300076789E42F2D18C4201D3002070BDA31C5E
:102340009BB2005D08B1401E00E0002080B210B1D9
:102350001C188C4201D9002070BD138070BD80F81C
:10236000301070472DE9F04104460D46002D26D06F
:102370002CB305F17800074601F05BF810B3002696
:10238000A6702C223946201DFEF780F884F83060B4
:10239000D5F8A4006063D5F8A800A0634FF6FF70DD
:1023A000A4F8240404F58260C4F82004C4F8266468
:1023B000A4F82A6484F82C64207828B107E00E2061
:1023C000BDE8F0810720FBE7FF2084F8540004F10A
:1023D00055010F46C4F810142046FFF75CFCA4F822
:1023E000140404F2144239462846FFF7F2FE00288E
:1023F000E6D104F23120C4F818042046FFF74BFC64
:10240000A4F81C0404F21C4205F13C00D4F8181492
:10241000FFF7DFFE0028D3D1012584F85150208B2F
:10242000A4F8480084F83C50266484F85060606941
:10243000606404F13C02002104F1540072DF0028C2
:10244000BED12570BCE7024608461188102906D087
:10245000112907D0262908D1114605F02BBC1146B9
:1024600005F017B9114605F07CBA70472DE9F04127
:1024700004460D462078002814D0A5700026C4F824
:102480002664A4F82A6484F82C64A079012708B192
:10249000012D0AD0E07908B1012D06D070B1022DCE
:1024A00003D00BE00820BDE8F081616B21B184F816
:1024B0002D740820884701E084F82D6429462046C1
:1024C000FFF7BBFBA070616B41B1032801D004286A
:1024D00004D1607910B194F82E0498B184F82F6477
:1024E00004F13C0018210546FDF7E9FF84F83C7033
:1024F00004F12C0005F074FC58B194F82C0084F819
:10250000510008E084F8306484F82F74072088476D
:10251000E6E784F8517094F8240058B104F12800DB
:1025200005F05EFC20B194F8280084F8520001E028
:1025300084F8527084F85060A07805281AD2DFE839
:1025400000F01703080D12002946204606F0EAF9AC
:1025500010E02946204606F0CDF90BE0294620463A
:1025600006F0F0F906E02946204606F016FA01E0EA
:1025700084F83160A07870B12A4604F15400D4F890
:10258000201472DF00288ED194F8301094F8540093
:1025900073DF002887D1616B11B194F8310088474F
:1025A000002080E72DE9F0410446002C12D01C22C7
:1025B00021461A48FDF76AFF1848194D0560206842
:1025C00058B17ADF002806D1206801682960406888
:1025D000686006E00E20BDE8F08111487BDF00282E
:1025E000F9D100240D4D4FF6FF76143DA5F12007DB
:1025F00004EB840005EB8000068007EB441141608A
:10260000084A0021001DFFF757FC08B10320E2E74C
:10261000641C002CECD00020DDE70000F435002025
:10262000902B0020B18F050010B50446204600F025
:1026300005F808B1204610BD142010BD142801D3A0
:10264000002070470146014802F089BE1436002080
:102650007CB505460C4620880930904201D90C20F3
:102660007CBD68466DDF0028FAD1218808206854B7
:102670002088401C80B220801B2129542088401CC7
:1026800080B220802844DDF801100160BDF80510FB
:1026900081802088801D80B220809DF8001049082C
:1026A00006D0012129542088401C208000207CBDB8
:1026B00000212954F7E70000F8B5044639483A4AA2
:1026C0003A4E2188801AC0087588212945D01ADC25
:1026D000354A344B4FF00300A3EB02024FEAD2021B
:1026E00000EB024010291DD011292FD0132933D11E
:1026F00000231A46852128467FDF00282CD0BDE81C
:10270000F840FFF7C7BB3B2942D0522935D05629A4
:1027100022D1A088132176DF00281DD0BDE8F84023
:10272000FFF7B8BB22A103F089FE072000F0F2FA00
:1027300008B1FFF7AFFBA1887180204802F056FF77
:10274000002809D0BDE8F840FFF7A4BB1CA103F0A6
:1027500075FE4FF6FF707080F8BD042101EB00405C
:102760001BA103F06BFE00200090A08869468FDF5C
:102770000028F1D0FFF78EFBF8BD00231A4619465A
:102780002846B1DF0028F7D0BDE8F840FFF782BB4C
:10279000A088132176DF0028EED0BDE8F840FFF7CF
:1027A00079BB000040A40500C0A30500E02A00207A
:1027B000436F6E6E65637465640000005C300020DA
:1027C000446973636F6E6E65637465640000000036
:1027D0005048592075706461746520726571756523
:1027E00073742E0010B5104C0188606810290FD04A
:1027F000112917D1401E6060002813D1FFF753FA4A
:1028000000280FD0216800290CD0BDE810400847EF
:1028100028B900F0DBFE10B1216801B1884760687B
:10282000401C606010BD0000882B0020018810292A
:1028300007D0112907D0122907D0502907D105F058
:1028400061BA04F0B9BE05F07BB804F099BE7047D8
:1028500070B50446A588208810280CD011281FD0F8
:10286000264B19283CD01A2846D1207A0409042C7A
:102870001BD301221AE005F00DFD284605F0E6FC09
:1028800048B1E07B022837D12946BDE870401B489B
:102890000C3802F06FBDBDE870400420FFF7FABAB3
:1028A0002846BDE8704005F019BD002229461846AB
:1028B00001F095F9032C01D3012200E000220F481A
:1028C0002946001F01F08BF9022C01D3012200E000
:1028D00000222946BDE870400848083801F07FB959
:1028E000207A002808D1607AC0F3C0022946BDE8EA
:1028F0007040184601F073B970BD00002836002002
:10290000F0B585B004460F4615461E46002C14D07F
:102910006A4631466069FFF733FC00280BD1A6F503
:102920007F40FF380BD0009848B1007848B1288824
:10293000F42808D9072005B0F0BD0E20FBE70520DC
:10294000F9E70820F7E70020019002900390049037
:10295000A088ADF804000497039501208DF80600C7
:1029600001A93046AEDFE6E770B58EB004463548C3
:1029700009AE90E82C00C0682CC60C90002C5DD0ED
:10298000E9B30868A061214609A862DF002853D195
:1029900020788DF836000125ADF83450A21C0DA921
:1029A0000120A8DF002847D1202101A8FDF787FDDD
:1029B0000220ADF8040020788DF80600F426ADF86A
:1029C0000860ADF80A508DF810509DF8110040F0E5
:1029D000080040F004008DF811008DF815508DF8B6
:1029E0001650608804F10C0201A900F01BFC0028BD
:1029F00022D1202101A8FDF762FD032000E01FE0A5
:102A0000ADF8040020788DF80600ADF80860ADF848
:102A10000A508DF810509DF8110040F010008DF80C
:102A200011008DF815508DF816508DF817506088EC
:102A3000221D01A900F0F6FB0EB070BD0E20FBE7D1
:102A40000E20F9E7A89605000246002912D0002AB8
:102A500010D008461188102906D0502907D05729D0
:102A600008D1114605F098B8114604F0DDBD1146B5
:102A700005F070B970470178407841EA002000F015
:102A80000100704708B504F05FF808B1FFF702FADB
:102A9000002000906946012003F0CCFE08B1FFF74A
:102AA000F9F9684603F05EFF002801D0FFF7F2F95C
:102AB00008BD00000749085C4FF0A04101F5A26184
:102AC0000968C14001F00100002800D0012080F019
:102AD00001007047649605007CB50024064E002571
:102AE0000323305D002200951146019503F022FA80
:102AF000641C032CF4D37CBD6496050010B5044619
:102B0000E00701D000F03CF8A00703D5BDE8104075
:102B1000FFF7E2BF10BD000007490B5C4FF0A04279
:102B200002F2045210680121994021EA0003536027
:102B30000140916070470000679605000249085CFB
:102B4000002103F062BA0000679605000249085CA4
:102B5000012103F05ABA0000679605000749085C96
:102B60004FF0A04101F204510968C14001F0010099
:102B7000002800D0012080F0010070476796050012
:102B80007CB50024084E0025305D0122009500230D
:102B90001146019503F0CEF9641C042CF4D3BDE872
:102BA0007C4000F003B800006796050010B50024D3
:102BB0002046FFF7C3FF641C042CF9D310BD10B5E9
:102BC00000242046FFF7C2FF641C042CF9D310BD7B
:102BD00010B501464FF0FF340020054A135C8B42CC
:102BE00001D1044602E0401C0328F7D3204610BD63
:102BF0006496050070B5024608460024064D2A601A
:102C0000002801D005F0A4FF686810B9FFF74BF861
:102C10000446204670BD0000882B00202DE9F047B7
:102C200081460E4600254846FFF7D2FF0446204F56
:102C3000032C31D21F4BDFF880A007F10308D6B177
:102C4000012E02D0022E27D122E004EB44001AF814
:102C5000005000EB0A06707848B1154A4FF48041E5
:102C6000921C5868FFF76CF908B987F80290B078A1
:102C700008F8040010E05868FFF78AF904EB4400F4
:102C8000504418F804108078814205D1054603E0CD
:102C900004EB440050444578002D06D0F968002923
:102CA00003D02846BDE8F0470847BDE8F08700009C
:102CB000102B00206C960500B0350020032801D2AF
:102CC000FFF7F8BE002070477047000030B503469C
:102CD0000020032B19D2012A02D101290BD0002296
:102CE0000B4D03EB43035C1969B1012907D002299D
:102CF00007D0072030BD03F10E02D2B2F0E7EA544C
:102D000030BD627030BDA27030BD072030BD000004
:102D1000B0350020024600200349097AC90702D0D5
:102D2000104600F059B87047102B002070B50646C9
:102D3000002424488660C160B00734D5002506E031
:102D4000012211462846FFF7C1FF04466D1C032DE2
:102D500001D2002CF4D034B940F2333203211A48A6
:102D6000FFF718F8044614B9FFF702F80446D4B97F
:102D70001548164A00210838FFF79EF81248144AF1
:102D80000121001FFFF798F808B1FFF783F80E48FC
:102D900000220C38A4218068FFF7D2F804462046B0
:102DA00008B1FFF777F8F0070AD00120FFF7A6FE79
:102DB00034B90548074A00210C38FFF77DF804466E
:102DC000204670BD102B0020789605006531050067
:102DD00009480500B14505002DE9F05F04460027CC
:102DE000854D00206978002902D0687001F0DEFB73
:102DF000824E01204FF47A694FF4C87840F2666A37
:102E00004FF4005B182C14D2DFE804F00C14143DCE
:102E10005E7F939EA3AEB9C4CFF3F3F3F3F3D3D79E
:102E2000DEE5F0F001F0C2FB3068FFF7B1F80746CD
:102E30002C70DEE00020FFF791FE40B10020FFF78C
:102E40007DFE022C01D14FF4E169C84606E0002066
:102E5000FFF77CFE022C01D14FF0C8082C704FEA1E
:102E6000C8304FF47A724FEA5841801841F100019E
:102E700052000023FDF7B6FA014600223068FFF742
:102E80005FF80746B5E00020FFF768FE28B1002094
:102E9000FFF754FE4FF4487003E00020FFF756FEA2
:102EA000C8202C70410CC0034FF47A72801841F195
:102EB000000152000023FDF795FA01460022306818
:102EC000FFF73EF8074694E00020FFF747FE20B1E9
:102ED0000020FFF733FEC84602E00020FFF736FE71
:102EE0002C704FEAC8304FF47A724FEA584180187C
:102EF00041F1000152000023FDF774FA014600225F
:102F00003068FFF71DF8074673E00020FFF726FE44
:102F100018B10020FFF712FE02E00020FFF716FEB6
:102F20002C7040F6CD4100223068FFF709F80746C3
:102F30005FE00020FFF7F0FD2C7000225146306862
:102F4000FEF7FEFF074654E00020FFF7FFFD2C7060
:102F50004FE068700120FFF7DFFD00225146306826
:102F6000FEF7EEFF074644E068700120FFF7D4FD4E
:102F7000002259463068FEF7E3FF074639E06870E3
:102F80000120FFF7C9FD002251463068FEF7D8FF47
:102F900007462EE068700120FFF7BEFD002259466B
:102FA0003068FEF7CDFF074623E0FFF708FE2C70E0
:102FB0001FE001F0FBFA2C701BE001F0F7FA002093
:102FC000FFF7C4FD2C7014E001F0F0FA0120FFF7C8
:102FD000BDFD2C700DE001F0E9FA0020FFF7B6FD11
:102FE0000120FFF7B3FD2C7003E0FFE7FFF7E7FDDB
:102FF0002C703846BDE8F09F102B00206C96050021
:1030000030B5002308E0C45CCD5CAC4202D05B1C50
:10301000D8B230BD5B1CDBB29342F4D3002030BD8C
:1030200070B505460C462046FDF770FAC2B2002086
:1030300008E0295C235C994202D0401CC0B270BDFC
:10304000401CC0B29042F4D3002070BD2DE9FC5F5B
:1030500005460F469346AC1C4FF001084FF000099F
:10306000CDF8049001A8FEF7B5FF204E70683860D7
:10307000D6E901011E4F401A3968081A401C06F2B1
:103080001C4A0FE00121504602F087F901F0BAFA1C
:103090000146504602F081F9D6E90101401A39682B
:1030A000081A401C8442EDD8B8F1000F17D0CDF8B3
:1030B0000090BBF1000F04D0052065F3891000904B
:1030C00003E0062065F39F5000907068396808405F
:1030D00006EB80000099C1607068204470609DF824
:1030E0000400FEF799FF4046BDE8FC9F6C390020C4
:1030F0003C2C002070B504460D460A2D03D10D214D
:103100002046FFF7F7FFA068411CA16021680D541D
:10311000D4E90110884204D32046BDE8704002F093
:103120001ABB70BD044881684068814201D101200A
:1031300070470020704700006C39002030B502460F
:10314000002107480478436805E003EBC1000578D7
:10315000954203D0491CA142F7DB002030BD00009E
:10316000C02B002000780221FFF758BD38B5044677
:103170000B490320FFF7DAFD08B1FEF78BFE694625
:103180000020FFF737FD08B1FEF784FE9DF8000030
:10319000022802D00020207038BD0120FBE700008B
:1031A000C92C050005494FF0FF3241F820200828BE
:1031B00002D3084480F8482070470000A036002061
:1031C000F0B507464FF0FF30002A02D04FF0000361
:1031D00001E04FF0080302D04FF0080501E04FF086
:1031E0000C050B4C04E054F82360761C03D05B1CE8
:1031F000AB42F8D3F0BDE51958B285F8300044F879
:103200002310002AF6D1E11881F84870F0BD0000C3
:10321000A03600200249084490F9300070470000B1
:10322000A03600202DE9F04391B006460C46154625
:10323000A078002818D08DF812002088ADF8100072
:1032400000270397607C03A905F0D1FBA07C0DF15A
:103250000C080DF10D0105F0CAFBE07B40B19DF8B3
:103260000E0040F0080107E001208DF81200E4E7AD
:103270009DF80E0020F008018DF80E10207C10B192
:1032800041F0100101E021F010018DF80E10207BBB
:1032900010B141F0010101E021F001018DF80E10A3
:1032A000207D08B1022000E0012060F342018DF88A
:1032B0000E101C210AA8FDF702F9607BC10601D49B
:1032C00080061AD50197E07C0DF104090DF1050186
:1032D00005F08DFB9DF8040020F00F00401C20F04D
:1032E000F00010308DF804009DF8060020F0060074
:1032F000801C8DF80600CDF83C90607B8DF828008E
:10330000A07B8DF82900142105A8FDF7D8F804A8A2
:103310000590CDF81880A088ADF82000A06820B1F5
:10332000E088ADF81C00A0680990A069A0B30297DE
:103330000088ADF83000A0694088ADF83200A0697F
:1033400040680B9002AF0E97A06902A9007B05F0C0
:103350004EFBA069791C407B05F049FBA069807A8F
:1033600020B19DF80A0040F0080103E09DF80A0032
:1033700020F008018DF80A10A069C07A10B141F060
:10338000100101E021F010018DF80A10A069007A07
:1033900018B141F0010002E00DE021F001008DF8CC
:1033A0000A00A169897B09B1022100E0012161F3D2
:1033B00042008DF80A00E06900B10D902B4605AA85
:1033C0000AA93046AADF11B0BDE8F08370B5054602
:1033D000002D01D0064C05E0054C083C02E0416898
:1033E00028468847204600F0FFFF0028F7D170BD2F
:1033F0009C36002070B504460126074D002C02D1F2
:103400006E70FFF7E3FF012C05D1AE70BDE8704090
:103410000120FFF7DBBF70BD8C360020D0E902230E
:10342000D1E90201801A994101D30120704700209F
:1034300070478178012903D190F82010012907D025
:10344000816A042906D0406A042803D0012070470D
:10345000002070470020704773B58CB006460020EE
:1034600001900D9800280FD0002401AD21460DA831
:1034700001F075FF28B10198411C05EB4000019156
:103480008480641C142CF1D32C2201A93046FCF753
:10349000FDFF0EB070BD0188062907D34FF44863C5
:1034A0004FF6FF72994203D9914201D0072070472D
:1034B0004088062803D3984203D9904201D00720C0
:1034C0007047914205D0904203D0814201D9072034
:1034D00070470020704770B506460D461446208898
:1034E000801D984201D90C2070BD3046FFF7D3FFF4
:1034F0000028F9D12188052068542088401C80B21A
:103500002080122129542088401C80B2208041193B
:10351000308805F0DFFC2188084480B22080411902
:10352000708805F0D7FC218808442080002070BDF9
:10353000FEF7B0BC00B587B01C216846FCF7BFFFA2
:10354000002000904FF4A03101914FF4F02102913E
:1035500003218DF80C10ADF80E008DF81000064810
:103560000590064806906846FFF71CF8002801D031
:10357000FEF790FC07B000BD65750500313505000C
:1035800038B54A7A104B002A0CD000220A725969C9
:10359000002906D001228DF80020ADF8020068460F
:1035A000884738BD0A7A62B19B684C680246194662
:1035B0002046FEF7C5FC0028F3D0BDE8384005F0F2
:1035C000E9B85B68F1E70000F435002010B5002190
:1035D00001220846FFF77AFB08B1072810D107221D
:1035E00002210120FFF772FB08B1072808D104224D
:1035F00002210020FFF76AFB08B1072800D1002054
:1036000010BD00007FB506460D461E481E493346D4
:10361000401AC408042000EB04402A461BA102F013
:1036200018FF002002900390ADF80850ADF80A5042
:10363000009001906A4602A9304690DF05462800B6
:103640001DD003F073FB0346012000EB0444324617
:103650001A49204602F0FDFEBDF8002012B9BDF85F
:10366000020028B1BDF80230204615A102F0F1FE9B
:10367000BDF804201AB12046214902F0E3FE04B04F
:10368000284670BDC0A30500C0A305005570646145
:1036900074696E672064617461206C656E6774681C
:1036A00020746F202575206F6E20636F6E6E6563CA
:1036B00074696F6E20307825782E0000C89A050056
:1036C000546865207265717565737465642054581B
:1036D0002F5258207061636B6574206C656E67743F
:1036E0006820697320746F6F206C6F6E6720627939
:1036F0002025752F2575206F63746574732E000067
:10370000149B050070B500240F4E10E0706800EBAC
:10371000C405287803F028FC6978012901D001212B
:1037200000E000214140287800F0D8F9641C30788E
:103730008442EBDBD6E90401084303D0BDE87040C6
:1037400005F068BB70BD0000C02B002010B5002143
:10375000024801F038FE80F3100010BD883D0020C3
:103760000A464FF48031914000F0A8B94FF4A0729E
:1037700002EB810189B200F027BA2DE9F04104463D
:103780000E4698464FF48035B5404FF4A07000EBDC
:10379000860081B222F07F472068C0F80853206875
:1037A000C0F84853206803F00FF8206800EB86004B
:1037B000C0F840752068C0F84453B8F1000F02D03B
:1037C0002068C0F80453BDE8F0810068D0F8040513
:1037D0007047000070B54379224C44F823204279A9
:1037E000241D04EBC2021279002A0CD008241E48C2
:1037F0001E49401AC008022101EB00401CA102F042
:103800001DFE204670BD0B880268C2F8083590F98D
:1038100004208978002A05DB02F1E022490182F8C0
:10382000001406E002F00F0202F1E022490182F8E2
:10383000141D90F904100125002909DB01F01F0374
:1038400005FA03F24909890001F1E021C1F80021DC
:10385000417904EBC1010D71417944F83100002038
:1038600070BD00001C2C002028A40500C0A305008A
:1038700052544320696E7374616E636520616C728B
:103880006561647920696E697469616C697A6564DF
:103890002E00000090F90400002809DB00F01F0250
:1038A000012191404009800000F1E020C0F80012A1
:1038B00070470A46022100F008B94FF4827100F007
:1038C00083B90068012101607047006801214160EF
:1038D00070472DE9F05F04460D4699464FF4803855
:1038E00008FA05F84FF4A07000EB85001FFA80FA83
:1038F00022F07F464146204600F0E0F82068D0F8EC
:10390000047500EB8500D0F840B5C0F8407551460D
:10391000206802F059FF3946584605F0D0F90128D1
:1039200006D1102003F05EFA5146206802F04CFFE9
:103930002068D0F804753046394605F0C0F9216892
:10394000C1F84483012814D0206800EB8500C0F83A
:1039500040652068D0F80475701E394605F0AFF94F
:103960006FF07F41A1EB0901814212D20D20BDE829
:10397000F09F2068761C00EB8500C0F840651020A1
:1039800003F030FA2068D0F80405B8420FD00D20BB
:10399000EDE760B92068761C00EB8500C0F8406553
:1039A0002068D0F80405B84201D00D20DFE70122DD
:1039B0004146204600F089F80020D8E72DE9F84379
:1039C00006460F46904699460F4D6946286801F015
:1039D00089FC0446ACB11C212046FCF770FD012097
:1039E00020712660C4F80890380BE060C4F8148099
:1039F0006946286801F09DFC04F0B0FB0020BDE89A
:103A0000F8830420FBE7000098990500D0E9031033
:103A1000084428DF7047000070B505460D4CE1688A
:103A2000002916D0080B0003E0600B4805F092FB5C
:103A300000232A460848E16801F062FF08B1FEF75A
:103A400029FA8623054A06490020FDF73BFB0020A2
:103A5000E06070BD9C2C0020402F0020CC99050018
:103A600034A2050030B587B004460D462068806852
:103A7000002821D0182101A8FCF721FD0295A0689B
:103A80000690207910B1012812D109E001208DF8AB
:103A9000040020690390E06804906069059007E0E5
:103AA00002208DF80400E06800030390606905902F
:103AB0002068816801A8884707B030BD0268C2F855
:103AC00048130068C0F8081370470368C3F844132C
:103AD000002A02D00068C0F8041370472DE9F84F9F
:103AE00082460E46504605F047F880464FF00009E2
:103AF000524601204946FCF7A6FC324F04460D46CB
:103B0000B8F1050F19D2DFE808F0031A23343C009E
:103B1000002E12D00121504605F03CF8CDF800905F
:103B20006846FEF757FAD7E9040104430D43C7E995
:103B300004459DF80000FEF76FFABDE8F88F0EB15E
:103B4000022100E000215046BDE8F84F05F022B800
:103B50004EB10321504605F01DF85046BDE8F84F20
:103B6000012105F078BA5046BDE8F84F012105F073
:103B700011B8002EE1D15046BDE8F84F042105F000
:103B800009B82EB15046BDE8F84F032105F002B840
:103B90000021504604F0FEFF0021504605F05BFA7C
:103BA000CDF800906846FEF715FAD7E9043223EA0B
:103BB000040022EA0501C7E904019DF80000FEF7B0
:103BC0002BFABAE7C02B002010B500684258002A33
:103BD00003D002F0F9FD012010BD002010BD002A25
:103BE00001D001F0C7BB01F0AFBB30B51488E51CB4
:103BF0009D4201D90C2030BD02230B5513885B1C5C
:103C00009BB213800124CC5413885B1C9BB213809D
:103C1000C8541088401C1080002030BD70B5044688
:103C20000D46B4F814140122D4F81004FEF75EFB1C
:103C300000B1057004F13C0204F5826104F1540006
:103C400072DF70BD2DE9F041464D47484749AB78DA
:103C5000401A0322C0080127002602EB0044012B72
:103C600007D02946022B08784A690ED0032B17D0BB
:103C700035E04FF4A020E8602F702869FFF7CCFEF4
:103C8000A878401CA8706E6129E0002827D1204642
:103C900037A102F0DEFB6E61A878401CA8701EE020
:103CA0000A326A61D8B9B2F5077F18DD204637A11C
:103CB000EB6902F0CEFBAA883DA14148EB69FDF714
:103CC000B1FD3F48FCF722FCC1B23D48FDF744F886
:103CD00020463B4A3BA102F0B5FBE8696E6168787B
:103CE000002823D0012815D0022821D003282FD066
:103CF00004281BD12878002818D1BFF34F8F3748EC
:103D00000168374A01F4E06111430160BFF34F8F4E
:103D100000BFFDE768690A3068618C2806DD20462F
:103D200030A102F08BFB6878401C6870BDE8F08120
:103D3000204631A102F082FB2F704FF49E20E860F4
:103D40000120FFF769FE6878401C68706E61EDE73E
:103D500068690A30686128780028E7D10420687013
:103D60006E61E3E79C2C002040A40500C0A3050081
:103D700065726173655F74696D65723D20256420AD
:103D8000206961705F663D202564200057524954C8
:103D9000455F5F74696D65723D20256420666C61C6
:103DA00073685F646F776E5F6E3D2025640000006E
:103DB000543D242646474E3D25642C2564000000D2
:103DC00000410020504F52545F73656E20645F6461
:103DD0006174613D20257320000000000CED00E0BF
:103DE0000400FA056C6173685F745F74696D6572D5
:103DF000203E203534300000696E5F6F75745F6956
:103E00006170202065726173655F666C6173685FC5
:103E1000616464722000000070B51349134A43685E
:103E2000891AC908032202EB0144002B05D0204661
:103E3000BDE870400EA102F001BB01780025184ECC
:103E4000012909D0022906D183680269204615A1FB
:103E500002F0FFFA357070BD83680269204617A131
:103E600002F0F7FA357070BD40A40500C0A305004C
:103E7000204552524F52207768696C6520657865FD
:103E8000637574696E6720616E206673746F72610A
:103E90006765206F7065726174696F6E2E00000037
:103EA0009C2C00202045524153455F524553554CB0
:103EB0005420256420307825782E00002057524960
:103EC00054455F524553554C542025642062307848
:103ED00025782E0010B596B09DF84C0020F00F000C
:103EE000401C20F0F0001030139000248DF80C409E
:103EF0004FF08050016E01910199406E084401908D
:103F0000019842F20F71B0FBF1F201FB1200019037
:103F100012A215A103A8019BFDF784FC03A8FCF7DE
:103F2000F5FA82B203A913A87CDF08B1FDF7B2FF4E
:103F3000149415941020ADF850003C20ADF85200B8
:103F4000ADF854404FF4C870ADF8560014A87ADFAD
:103F5000002801D0FDF79EFF16B010BD59535F44F5
:103F6000616D70657200000025732D25303464008A
:103F70002DE9F04104461D4F48887A88904232D19D
:103F80000888A0F52062773A2DD18888C01E82B2B9
:103F9000BA80174817491346401AC508032000EB9A
:103FA000054015A102F055FA1A4B02201880002195
:103FB000B8884FF6FF761A8806EA42021A808242D3
:103FC00003D318884008188003E0491CC9B20829A7
:103FD000F1D304202388628800EB0540BDE8F0415E
:103FE0000DA102F036BABDE8F0810000E02A002001
:103FF00040A40500C0A3050044617461206C656E97
:104000002069732073657420746F203078255828D8
:1040100025642900A02C0020415454204D545520E3
:1040200065786368616E676520636F6D706C657439
:1040300065642E2063656E7472616C20307825781B
:10404000207065726970686572616C2030782578BF
:104050000000000010B50949094801F038FA08B11C
:10406000FDF718FFF721064801F024FA002803D0D5
:10407000BDE81040FDF70EBF10BD0000713F050008
:104080004830002010B50B48FFF79FFB094A083A5B
:10409000D2E90434C01844F10001D2E90632C31A4F
:1040A00071EB020204D24FF08072801841F10001DE
:1040B00010BD0000002C002010B5C0B2FFF73EF884
:1040C0000446207802F050FF01466078012801D0B4
:1040D000012000E000204840002808D00448D0E932
:1040E0000410014303D1BDE8104004F093BE10BD9D
:1040F000C02B002030B50546002000220EE0000154
:10410000AB5CA3F13004092C01D8204304E0413B0F
:10411000052B01D80A331843521CD2B28A42EED37F
:1041200030BD000038B514490022144801F088FC65
:1041300008B1FDF7AFFE4FF49E240423104A214638
:104140000E4801F0EFFC0E4808388268521C0ED170
:104150000C4A826001220270002000900423084A69
:104160002146064801F0EAFD08B1FDF793FEBDE8DF
:104170003840024803F042BFA8990500402F0020B4
:10418000A42C0020FE0FDCBA10B50C4A01210C480B
:10419000FDF792FE08B1FDF77DFE0A490020487048
:1041A00007480022A4210068FDF7CAFE002803D0BA
:1041B000BDE81040FDF76EBE10BD0000453C050097
:1041C000C89905009C2C002010B50A4941600A4896
:1041D00001F0E0F858B902F005FD074908740548F8
:1041E0001C23001F8C228C39006801F067F8002026
:1041F00010BD00009C990500B04000200021084A35
:1042000001EB810332F82330834204D101EB8100BA
:1042100002EB80007047491C0029F1D00020704754
:10422000E03500202DE9FC5F8346DDE90C470E46B2
:1042300091469846C6F1000A002E01DA504600E089
:104240003046012502E090FBF9F06D1C4845FADA92
:10425000A84500D9454624B1002E01DB780700D5DA
:10426000641EB80702D5B8F1000F0BD0F80709D1CA
:104270002CB907E0641E20215846FEF73BFF0CB125
:10428000A542F7D3002E05DA56462D215846FEF7F3
:1042900031FF05E0780703D52B215846FEF72AFFAA
:1042A00007F0030002280CD1B8F1000F09D12CB996
:1042B00007E0641E30215846FEF71CFF0CB1A542F2
:1042C000F7D3CDE9004743464A463146584604F005
:1042D00017FEBDE8FC9F024600201268530714D564
:1042E00002F00300012802D002280DD106E0C2F33B
:1042F00083100B68801C1844086005E002230868DE
:1043000003EB925210440860012070472DE9F04100
:1043100006460F46904600241BE0204602F010FDA2
:1043200005464FF48031A1402846305800B10120A5
:1043300068B1D6F80403084000D0012038B12946FE
:10434000304602F003FDD7E9002128469047641C5F
:10435000E4B24445E1D3BDE8F08100000121814091
:1043600003484068014201D0012070470020704797
:10437000A82B0020014601208840FDF789BE0000DF
:104380000248007A002800D001207047B040002089
:10439000F0B58488A618944200D82246A71AC5888A
:1043A000EC189D4200D82B46EB1A4A880588AA4291
:1043B00002D34088824201D90020F0BD8888B842EB
:1043C00001D3B04201D90020F0BDC888984201D382
:1043D000A04201D90020F0BD0120F0BD01218140A3
:1043E000C80300D00120704701460868002801D0AA
:1043F00002680A60704710B5044622460121002079
:1044000001F0D4FD002154F821300BB1012010BD82
:10441000491C0029F7D0002010BD00002DE9F0470D
:104420005E486E215E4B00780A220027DFF8749107
:104430004FF4FA744FF4967500281DD0C9F8404027
:10444000C9F8445053F82000192390FBF3F0C9F841
:104450000470C9F80820C9F81870C9F81C20C9F8F8
:104460002C70C9F83020012840D0022843D00328FE
:1044700046D0042849D054E0C9F80440C9F808508F
:10448000186832380C2390FBF3F0C9F81870C9F89B
:104490001C20C9F82C70C9F83020C9F84070C9F840
:1044A0004420012806D0022809D003280CD0042873
:1044B0000FD036E0C9F81810C9F81C7031E0C9F8FF
:1044C0002C10C9F830702CE0C9F84010C9F84470BD
:1044D00027E0C9F81810C9F81C70C9F82C10C9F8E1
:1044E0003070C9F84010C9F844701AE0C9F80410D7
:1044F000C9F8087015E0C9F81810C9F81C7010E068
:10450000C9F82C10C9F830700BE0C9F80410C9F8CC
:104510000870C9F81810C9F81C70C9F82C10C9F82F
:1045200030700025DFF8808005EB850409EB8406F8
:10453000F068012819D059F824000A3049F82400FD
:10454000B06818B118F80500FEF7F8FA59F8240019
:10455000B168884203DD49F824700120F0606D1CC9
:10456000EDB2042DE0D3BDE8F087706848B159F88A
:1045700024000A3049F8240018F80500FEF7E6FA8E
:1045800003E018F80500FEF7D9FA59F8240071681D
:104590008842E4DD49F82470F760E0E7302F00201E
:1045A000182F00208C430020F4990500FEF7FEBA76
:1045B0007047000010B502F0CFFB002804D102F0D4
:1045C000F9FB02490020887010BD00008C360020E5
:1045D000F721018017214180002101714171FB21E8
:1045E00081711B21C171704710B54FF480410020CB
:1045F00001F098FF08B1FDF74DFCBDE8104001F057
:10460000DDBD00002DE9FF410025264800F0BFFE7A
:104610002448001F074600F0BAFE234EB0680390FE
:1046200022490C68204006EB80000C3003A9FFF7FC
:1046300052FE28B10398204006EB80000C30F5E7CD
:1046400000206B4603994A1C214006EB810103922E
:10465000C96843F82010401C0228F3D3009800F0EA
:10466000030001280CD0022812D1BDF80650009892
:10467000032101EB9050039901EB9000039007E0B8
:10468000BDF8065000980399C0F3831008440390C6
:10469000384600F079FE08B10398B06004B02846AF
:1046A000BDE8F081843D00206C3900203C2C0020C6
:1046B00086B04A48D0E907238169406ACDE90223E0
:1046C00001910490FFF790FF04F0B0FB05A8FEF7FE
:1046D0004DFDFEF76BFA03F037FC0120FEF736FACA
:1046E000FEF7D0F90020FEF731FAFFF7F3FB0220C6
:1046F000FEF72CFAFFF7AEFC0320FEF727FA04F0D2
:10470000DBF8FDF7EBFAFEF715FF35483549401A9F
:10471000C008032101EB004033A101F08FFE01F03E
:104720005BFD0028FBD1082001F028FC0B2001F0E4
:1047300025FC0021082001F05CFC00210B2001F089
:1047400058FC0C2001F01AFC0D2001F017FC0E2083
:1047500001F014FC0F2001F011FC102001F00EFC00
:10476000112001F00BFC122001F008FC01210C20AB
:1047700001F03FFC01210D2001F03BFC01210E2046
:1047800001F037FC01210F2001F033FC0121102042
:1047900001F02FFC0121112001F02BFC012112203E
:1047A00001F027FCFDF7D6FA0020FEF7C7F901203B
:1047B000FEF7C4F90220FEF7C1F9FEF7F7F903F09E
:1047C0008FFEFFF7AFFCFFF7DFFC01F0CDFF01F03C
:1047D00003FD0028FBD102F037FEF6E7F491050057
:1047E00040A40500C0A305004465627567206C6F96
:1047F0006767696E6720666F722061707020206144
:104800007070382D343800002DE9F047484C20698D
:10481000401C2061FCF76EFAFFF700FE20690521BD
:1048200090FBF1F201FB120000287FD1DFF8049128
:104830000C27002699F809003F4C404D4FF019080D
:10484000022801D004282DD189F809602A78002A8D
:104850000DD054F8220000F1190044F8220054F859
:10486000220009D1A0F1320090FBF7F306E02068A6
:1048700000F10C002060F2E790FBF8F303F1010374
:10488000012B01DA012302E0052B00DD05232CA119
:104890002F48FCF7C7FF2E48FBF738FEC1B22C4863
:1048A000FCF75AFA2B49487A022801D0042804D18F
:1048B0004E722878C0F1010028702749487A0228F2
:1048C00001D0042832D14E7289F809602A78002A72
:1048D0000DD054F82200A0F1190044F8220054F839
:1048E000220009D1A0F1320090FBF7F306E0206826
:1048F000A0F10C002060F2E790FBF8F303F1010354
:10490000012B01DA012302E0052B00DD05230CA1B8
:104910000F48FCF787FF0E48FBF7F8FDBDE8F047AE
:10492000C1B20B4800E001E0FCF716BABDE8F08721
:10493000102B002000430020182F0020302F0020D3
:10494000543D2426524D453D25642C25640000002D
:10495000004100200C4300201843002070B505469C
:104960000E461446A888801C2188821C0A449A425C
:1049700001D90C2070BDFE2801D90C2070BD401C4F
:1049800070542088401C80B22080FF213154208840
:10499000401C80B220808119288804F09BFA21886D
:1049A000084480B22080AA8842B1A96841B130444D
:1049B000FBF76CFD2088A98808442080002070BD8A
:1049C000072070BD2DE9F0478946DDF820A0054697
:1049D000C688407906FB00F73F1F181D0146B0FB53
:1049E000F6F0B1FBF6F406FB1411146804EB030CAB
:1049F000BC4500D9FC1A146001E02D68401E002857
:104A0000FBD18046771AA7421BD9274619E009EB4C
:104A100008036818001DBAF1000F05D001463A4698
:104A20001846FBF733FD03E03A461946FBF72EFD27
:104A300000212D68E41BB844A64201D9274600E0B6
:104A40003746002CE3D1BDE8F087000070B5FF22A7
:104A5000FF23084D05F5807605E010F8014B544022
:104A60002A5D5A40335D491E4C1CF6D142EA0320B0
:104A700070BD0000CD2C002030B50446002912D0B6
:104A800001F064FD0021094B09E003EB8102256878
:104A90001288AA4202D12160002030BD491C814207
:104AA000F3D3052030BD002030BD00000000000021
:104AB00070B5334D6868401C686029460978012943
:104AC00001D1401D686068681D2801DD0020686014
:104AD00000242B4E3836002256F82400002801DA34
:104AE000414200E001461D2906DD1F2391FBF3F141
:104AF0006B688B4200DA012214B1012C1ED03AE01F
:104B000052B1002811DD00210D2001F08AFA0121A7
:104B10000E2001F086FA2EE000210D2001F081FA2E
:104B200000210E2001F07DFA25E001210D2001F089
:104B300078FA00210E2001F074FA1CE052B100282E
:104B400011DD0121112001F06CFA0021122001F089
:104B500068FA10E00021112001F063FA0021122010
:104B600001F05FFA07E00021112001F05AFA01215B
:104B7000122001F056FA641C022CACD370BD000068
:104B8000F02E00202DE9F05F0024DFF8EC82BB4F0F
:104B900008F1280908F1300A08F13806B64818303B
:104BA000A0F1080250F8241052F82400081A42F824
:104BB00024104FF4FA73984202DDA0F57A7004E0F5
:104BC00010F5FA7F01DA00F57A70032290FBF2F11A
:104BD000A94DD5F808C0614401EBD1714910A96015
:104BE000D5F80CC00CF1010CC5F80CC018F804C0C5
:104BF000BCF1000F10D005F1200151F82420104421
:104C000041F82400002C6FD059F8240064286CDD92
:104C1000642049F824000DE104EB840517F825C051
:104C2000BCF1000F15D0BCF1010F34D0BCF1020F64
:104C30003DD0BCF1030F60D0BCF1040F6CD0BCF1CF
:104C4000050F7DD0BCF1060F7BD0BCF1070F79D0EA
:104C500008E18A488A49403800EB441B5846FCF773
:104C60001AF95846FCF72AF94FF42F60CAF80000E9
:104C700041F2CC00CAF804002CB117F82500401C02
:104C800007F82500EEE098F80100012802D13878F5
:104C9000401C3870E6E0002146F8241007EB850040
:104CA0004160C1600161022007F82500DAE0BCB173
:104CB0006FF04F0146F8241007EB85010B690344A0
:104CC0000B61CB681B1ACB604868C01C4860C828C1
:104CD00012DD40F6B830834208DA07F8252008E0F4
:104CE0006FF095013160E7E791E09EE0052007F85D
:104CF000250000204860C860B4E0002246F8242067
:104D000007EB85004168C91C4160642903DD4260EE
:104D1000042007F82500A5E046F8243007EB8501BC
:104D20000A6902440A61CA680244CA604868C01C31
:104D30004860C82811DD40F6B830824207DD02E045
:104D40000CE025E05FE0052007F8250002E00720E1
:104D500007F8250000204860C86083E0A4B16FF028
:104D6000310246F8242011F11E0F02DA062107F85D
:104D7000251007EB850100228A600A69104408614A
:104D80006FF00E0048606DE06FF095023260EAE768
:104D9000A4B33C4946F8241007EB85014B68DB1CA3
:104DA0004B608A68151A8D600A6902440A61D1F85D
:104DB0000CC0ACEB0000C860412B53DD00234B60FE
:104DC00040F6340C65450BDA012508F80450002A3A
:104DD00006DA52425AF8245092FBF5F249F82420A0
:104DE0008B605AF82410C1EB011101EB8101B0EB8B
:104DF000410F37DD012008F8040033E0FFE72149C7
:104E0000B4393160C8E7002046F824002AE0D9F818
:104E10000000642803DD6420C9F800000AE032289D
:104E200008DA3220C9F8000004E0002802DA002085
:104E300049F8240059F82400052800DA05205AF81A
:104E40002420424351F82400111A0C48403800EB4A
:104E50004410FBF7F5FFE96840F24B1291FBF2F3C7
:104E600046F82400641CE4B2022CFFF497AEFFF76E
:104E70001FFEBDE8F09F0000F02E002064430020DC
:104E8000E09905008EFEFFFFF8B505460F46144673
:104E90002978012901D1687830B12088821C9A4292
:104EA00009D8012902D008E00720F8BD697801443B
:104EB000891C994201D90C20F8BD181A801E86B2AF
:104EC00000962188B81C084469467DDF0028F3D18C
:104ED0002978022904D06878BDF80020904205D3D3
:104EE000BDF80000B04201D8092008E008200129DF
:104EF00004D16978B14201D8009100E00096BDF874
:104F00000010FE2901D90C20F8BD2288491CB95493
:104F10002188491C89B2218078542088401C208037
:104F2000BDF80010084420800020F8BD4FF08051EB
:104F3000D1F83001421C05D0D1F83411062809D02F
:104F4000002070470D4800780C4908310978C1F3FA
:104F50000311F3E7C91E05290ED2DFE801F00305AE
:104F600007090B000120704701207047012070479E
:104F7000012070470120704701207047E00F00F0CA
:104F80004FF08051D1F83001421C05D0D1F83411D6
:104F9000062809D0002070470D4800780C490831D8
:104FA0000978C1F30311F3E7C91E05290ED2DFE822
:104FB00001F0030507090B0001207047012070472D
:104FC0000120704701207047012070470120704781
:104FD000E00F00F04FF08051D1F83001421C05D0B5
:104FE000D1F83411062809D0002070470D48007808
:104FF0000C4908310978C1F30311F3E7C91E0529EB
:105000000ED2DFE801F0030507090B00012070470D
:105010000120704701207047012070470120704730
:1050200001207047E00F00F00F4801780E4808306B
:105030000078C0F30310062901D000207047C01E7D
:1050400005280ED2DFE800F0030507090B00012058
:1050500070470020704700207047002070470020F4
:105060007047002070470000E00F00F00D48016815
:105070004068062901D000207047C01E05280ED2C6
:10508000DFE800F0030507090B000020704700204F
:1050900070470020704701207047012070470120B1
:1050A00070470000300100100D4801684068062973
:1050B00001D000207047C01E05280ED2DFE800F0A6
:1050C000030507090B0000207047002070470020EF
:1050D0007047002070470120704701207047000092
:1050E000300100104FF08051D1F83001421C05D042
:1050F000D1F83411062809D0002070470D480078F7
:105100000C4908310978C1F30311F3E7C91E0529D9
:105110000ED2DFE801F0030507090B0001207047FC
:10512000012070470120704701207047012070471F
:1051300001207047E00F00F00F4801780E4808305A
:105140000078C0F30310062901D000207047C01E6C
:1051500005280ED2DFE800F0030507090B00012047
:1051600070470020704700207047002070470020E3
:105170007047002070470000E00F00F04FF08051B2
:10518000D1F83001421C05D0D1F83411062809D0DD
:10519000002070470D4800780C4908310978C1F3A8
:1051A0000311F3E7C91E05290ED2DFE801F003055C
:1051B00007090B000120704701207047012070474C
:1051C000012070470120704701207047E00F00F078
:1051D0000F4801780E4808300078C0F30310062904
:1051E00001D000207047C01E05280ED2DFE800F075
:1051F000030507090B0001207047002070470020BD
:105200007047002070470020704700207047000062
:10521000E00F00F00F4801780E4808300078C0F326
:105220000310062901D000207047C01E05280ED2A9
:10523000DFE800F0030507090B000120704700209C
:105240007047002070470020704700207047002002
:1052500070470000E00F00F04FF08051D1F83001AE
:10526000421C05D0D1F83411062809D0002070471F
:105270000D4800780C4908310978C1F30311F3E7B0
:10528000C91E05290ED2DFE801F0030507090B004E
:1052900000207047002070470120704701207047B0
:1052A0000120704701207047E00F00F010B5FAF7B9
:1052B000FCFF08B1002010BD112010BD10B5002961
:1052C00006D0B2FBF3F403FB14241CB1092010BD7B
:1052D0000E2010BD01600021416081608281C38188
:1052E000002010BD70B504460D4629462046FAF749
:1052F00091FF18B129882068084470BD002070BD56
:1053000010B50A8849888A4203D1FAF7C5FF0120FF
:1053100010BD002010BD70B504460D46294620463C
:10532000FAF79DFF18B169882068084470BD002015
:1053300070BD10B50A8849888A4203D1FAF786FF02
:10534000012010BD002010BD01F01F0301229A4072
:10535000D243490900EB8100114600F024B84A0904
:1053600050F8220001F01F0201219140084000D0B6
:10537000012070470A4602F01F030121994052099B
:1053800000EB820000F024B8002100F012B80121E7
:1053900000F01EB8012100F011B808B56A46FAF70E
:1053A000D0FF009808BD08B56A46FAF7B0FF00982C
:1053B00008BD08B56A46FAF7AAFF08BD08B56A46EF
:1053C000FAF798FF08BD08B56A46FAF787FF08BDE7
:1053D00008B56A46FAF78EFF009808BD08B56A4618
:1053E000FAF7BCFF009808BD38B504460025002038
:1053F00000906846FCF7EEFD2168626808689042FC
:105400000FD9401E08600178204600F02DF80546AF
:105410002068217A0278891AC9B202798A4200D2B8
:1054200001719DF80000FCF7F7FD284638BDC26801
:10543000008A891AB1FBF0F0C0B2704738B5054652
:105440000C46002000906846FCF7C4FD2146284623
:10545000FFF7EDFF2A6811684B1C136008709DF878
:105460000000FCF7D9FD38BDC268008A01FB0020AE
:10547000704710B5002806D0017A4268891AC9B26F
:1054800003681A6006E00E2010BD03681A68541CF9
:105490001C601170491EC9B2F7D200680021017169
:1054A000002010BDC20800F007030120895C98406D
:1054B00008407047002805D0A1F11702E12A03D364
:1054C000072070470E20704701800020704770B59C
:1054D0000546002D10D02961F72028806880FB2028
:1054E0002871002405EBC400801DFFF771F8641CCF
:1054F000002CF7D0002070BD0E2070BD70B50246A4
:105500000C469588002D50D11088242820D006DC28
:10551000102809D011280CD0232822D11DE03A28C8
:105520000CD055281DD10EE01146204602F0B8F8E7
:1055300017E01146204602F02EFA12E011462046EE
:1055400002F0D6FA0DE01146204602F02BFA08E0F0
:105550001146204602F02AF903E01146204602F0E7
:10556000AFF9A07A002820D0E1882846A5DF0F49AE
:105570000F4A0126891ACD0858B1112815D001F01B
:10558000D5FB024606EB0540BDE8704009A100F0DE
:1055900059BF0023A372E6720420E28800EB0540A5
:1055A000BDE87040104900F054BF70BDC0A30500B5
:1055B000C0A3050073645F626C655F6761747463A8
:1055C0005F65786368616E67655F6D74755F72654E
:1055D000717565737428292072657475726E6564BF
:1055E0002025732E00000000809A0500002804D0BA
:1055F0000278DE2A03D0082070470E2070474180D1
:105600000020704700280CD069B10278DE2A0CD047
:1056100009684160DE2101704FF6FF714180002072
:1056200070470E2070470E2070470820704770B5F5
:10563000044600292ED0002C2CD00D462878DE28D8
:1056400028D1A0886988884202D1284603F0EEFC60
:10565000208801280BD002280FD0112813D0512800
:1056600018D1211D2846BDE8704002F0F9BA211D6D
:105670002846BDE8704002F038BB211D2846BDE831
:10568000704002F031BBA0886988884202D14FF691
:10569000FF70688070BD00F180400068002800D075
:1056A0000120704708B500F18040002101600068CA
:1056B000009008BD70B50E4C01252078002801D05F
:1056C00085260EE00020A06060602061E06009484F
:1056D00001F060FB064601F085FA08B901F044FBD1
:1056E000257001F039FB00B1A570304670BD000097
:1056F0008C360020F533050008B500200090684680
:10570000FCF768FC0648C168491EC160C06808B95A
:10571000FEF750FF9DF80000FCF77EFC08BD00007E
:105720008C36002004480178002901D0852070477C
:105730000121017000207047B02B00200FB408B584
:105740000399002904D004AA00926A4600F00FF8D9
:1057500001B05DF814FB10B50446A268002A05D01C
:10576000D4E90403216898470020A06010BD2DE90A
:10577000FC4106460C461546002C75D014F8011B5A
:1057800039B125290DD03046FDF7B4FC207800282A
:10579000F4D1307B002867D03046BDE8FC41FFF7EC
:1057A000DABF0023012021782B291DD02D2913D009
:1057B000302915D000200028F5D100222A2917D041
:1057C0002178A1F130000A2818D2641C02EB820073
:1057D00001EB4002303AF1E743F00103641CEAE7D1
:1057E00043F00203641CE6E743F00403641CE2E7B1
:1057F0002868011D296000680244641C002021788B
:105800002E290CD1641C2178A1F130070A2F06D271
:10581000641C00EB800001EB40003038F3E76C299A
:105820000DD068290BD069291FD00BDC25295FD04A
:10583000582932D063290ED064295DD115E0641C4B
:105840002178ECE770293CD0732932D0752918D023
:10585000782951D121E02868011D29600078C1B262
:105860003046FDF747FC47E048E029680F1D2F60F0
:105870000968CDE9002303460A223046FEF7D2FC30
:105880003AE029680F1D2F600968CDE9002303461F
:105890000A22304603F034FB2EE029680F1D2F60EA
:1058A0000968CDE9002303461022304603F028FBA7
:1058B00022E02868011D29600168304603F0CAF91A
:1058C0001AE02868011D2960076830213046FDF77D
:1058D00011FC78213046FDF70DFC08210020CDE9B0
:1058E00000100B4610223946304603F009FB03E056
:1058F00025213046FDF7FEFB641C47E7BDE8FC812F
:105900002DE9F84305460F46164698462D482E4980
:10591000401AC008012101EB0044002D1FD0286867
:1059200040B3002E30D039462846FCF767F94FF0D7
:105930001009002832D06868394602682846724348
:10594000FCF76FF9002833D02868434632460469D3
:1059500001B039462846A446BDE8F04360470E2012
:1059600000902046194B1AA21BA100F07AFD0E20D0
:10597000BDE8F883082000902046144B21A216A110
:1059800000F06FFD0820F3E70920009020460F4B40
:105990001FA211A100F065FD0920E9E720460B4B8D
:1059A0001CA20DA1CDF8009000F05BFD1020DFE7F8
:1059B0002046064B214A08A1CDF8009000F051FD89
:1059C0001020D5E760A40500C0A305008399050059
:1059D000705F667300000000257320636865636B69
:1059E000206661696C656420696E20257328292012
:1059F000776974682076616C756520307825782E1B
:105A000000000000705F66732D3E705F617069007A
:105A10006C656E00616464725F69735F7061676575
:105A20005F616C69676E656428705F66732C2070B7
:105A30006167655F6164647229000000E4A105008C
:105A400038B503461148124C0E25001BC00801242E
:105A500004EB0040002B09D081B119600C6801B043
:105A6000A446BDE83040114618466047094B0AA2DB
:105A70000BA1009500F0F5FC0E2038BD054B13A2DC
:105A800007A1009500F0EDFC0E2038BD60A40500D4
:105A9000C0A3050038990500705F66730000000020
:105AA000257320636865636B206661696C6564209B
:105AB000696E202573282920776974682076616CC7
:105AC000756520307825782E00000000705F6170C9
:105AD000690000002DE9F041002805D0016819B1E6
:105AE000C969BDE8F041084700240C4E0C48851BED
:105AF00014270CE004EB840006EB8000016829B158
:105B0000C969884710B10120BDE8F081641CB5FB6C
:105B1000F7F0A042EED80020F6E70000402F00206A
:105B2000542F00202DE9F8430546884617461E46A7
:105B3000314A32480E21101AC008012202EB0044FB
:105B4000002D1ED03FB3286800282DD0002E35D060
:105B50004046FCF74DF84FF01009002838D0324687
:105B600041462846FCF75DF800283BD028683346BC
:105B70003A46846801B041462846A446BDE8F04351
:105B80006047009120461E4B1EA220A100F069FC38
:105B90000E20BDE8F88300912046194B26A21BA1D8
:105BA00000F05FFC0E20F4E7082000902046144B24
:105BB00023A216A100F055FC0820EAE70920009076
:105BC00020460F4B21A211A100F04BFC0920E0E779
:105BD00020460B4B1EA20DA1CDF8009000F041FC19
:105BE0001020D6E72046064B1FA208A1CDF8009052
:105BF00000F037FC1020CCE760A40500C0A305002E
:105C00005E990500705F66730000000025732063D5
:105C10006865636B206661696C656420696E202528
:105C200073282920776974682076616C7565203047
:105C30007825782E00000000705F646573740000A2
:105C4000705F66732D3E705F617069006C656E00F9
:105C5000616464725F69735F616C69676E65643308
:105C60003228737263290000616464725F69735F34
:105C700077697468696E5F626F756E647328705FB0
:105C800066732C207372632C206C656E29000000F3
:105C9000044801214174007A002801D00020704797
:105CA00001207047B0400020012801D0032808D10E
:105CB000044900224A74012800D00020087402F030
:105CC00015BA7047B040002070B50446022C01D0D0
:105CD000032C2DD1174D287A002829D001281BD05C
:105CE000022819D10020144E022C316802D0032C56
:105CF00007D103E0084601F081FF02E0084601F009
:105D00006FFF48B100202872022C0BD00D213068A3
:105D1000FDF7A8FE02F0CEF9687C28B1BDE870401E
:105D200000F066BF0021F2E7BDE8704002F0DEB986
:105D300070BD0000B0400020942C00202DE9F84FE9
:105D40000546DDF828908A4690461E463F48404A60
:105D50000E21801AC008012202EB0044002D1AD047
:105D6000B8F1000F20D02868002826D00921002E85
:105D70002DD068684068B6FBF0F200FB1260002886
:105D80002ED000912046334B33A23EA100F069FB98
:105D90000920BDE8F88F009120462E4B44A239A17E
:105DA00000F05FFB0E20F4E700912046294B42A251
:105DB00034A100F056FB0E20EBE7082000902046AF
:105DC000244B3FA22FA100F04CFB0820E1E70091FB
:105DD0002046204B3DA22BA100F043FB0920D8E731
:105DE0005046FBF705FF1027A0B14046FBF700FF28
:105DF000C8B1324651462846FBF713FF00281BD096
:105E0000CDF80090286833464246C468514628467B
:105E1000A047BEE720460F4B2DA21AA1009700F025
:105E200020FB1020B5E720460A4B2FA215A10097B2
:105E300000F017FB1020ACE72046064B33A211A15F
:105E4000009700F00EFB1020A3E7000060A40500FF
:105E5000C0A305007099050021286C656E202520DF
:105E6000705F66732D3E705F666C6173685F696E0C
:105E7000666F2D3E70726F6772616D5F756E6974CB
:105E800029000000257320636865636B20666169E3
:105E90006C656420696E20257328292077697468F1
:105EA0002076616C756520307825782E0000000022
:105EB000705F667300000000705F73726300000023
:105EC000705F66732D3E705F617069006C656E0077
:105ED000616464725F69735F616C69676E65643386
:105EE0003228646573742900616464725F69735F4A
:105EF000616C69676E65643332282875696E743326
:105F0000325F7429705F7372632900006164647288
:105F10005F69735F77697468696E5F626F756E64DD
:105F20007328705F66732C20646573742C206C6515
:105F30006E29000070B5DDE904654FF0A04441EA28
:105F4000420141EA830141EA062104EB800041EA73
:105F50000541C0F8001770BD70B5DDE904654FF06C
:105F6000A04441EA420141EA830141EA062104EBEF
:105F7000800041EA0541C0F8001770BD4FF0A04213
:105F800002EB80000321C0F8001770474FF0A042D9
:105F900002EB800000F5E060026822F4403202600B
:105FA000026842EA014101607047000038B5084BC1
:105FB0001B6800936C46451807E054F82030D3F86E
:105FC000201502C2C3F82015401C8542F5D838BD03
:105FD000B896050042090021002A00D1491E00F0B0
:105FE0001F00012282400A4201D001207047002098
:105FF0007047012282404FF0A043002902D0C3F82D
:1060000008257047C3F80C257047012282404FF0E5
:10601000A043002902D0C3F808257047C3F80C2517
:106020007047012282404FF0A043002902D0C3F8FC
:1060300008257047C3F80C257047000008B50349D0
:106040000844002101600068009008BD0060004025
:10605000034908440068012800D000207047000070
:106060000060004010B50446FCF770F8411C0DD0EC
:10607000E1680871094AD2F8101441B1C968E368AF
:1060800009681960D2F81014C9680C6010BDC2F814
:106090001044E2680021116010BD00006C3900203E
:1060A0007047FAF7B9BF704708B5034A009240231A
:1060B000024A00F005F808BDC5870500D437002066
:1060C000F0B593B00F46189E14461D46384600F0B2
:1060D00012FB18210DA8FAF7F2F90D940E951296FD
:1060E0000023082207A9384600F01AFB0826099861
:1060F0000A90BDF82000ADF82C00BDF82200ADF8E4
:106100002E0000208DF83100079800F003000128D0
:1061100002D0022819D034E00798850A0798C0F306
:10612000C2008DF830000798C0F38314A2003346F4
:1061300001A9384600F0F4FA0DA800900AAB2246F7
:1061400001A9284600F030FA1BE00798840D079853
:10615000C0F3C2008DF83000082C01D2254600E0C3
:10616000082533462A4605A9384600F0D9FA2E44B8
:10617000641B0DAB0AAA294605A800F07DF9002C86
:10618000EAD1384600F0BDFA13B0F0BD0A4A02EB7E
:10619000C000012907D0022907D0032907D004290C
:1061A00007D0002070470220704704207047007914
:1061B0007047407970470000C0A3050010B5FFF795
:1061C00070FF04210348FFF74DFF02490120C96811
:1061D000487110BDB0A305002DE9F04F85B0FCF764
:1061E000A1FF18B1002005B0BDE8F08F894F4FF036
:1061F0000008C7F81884BFF34F8FB8680490864929
:106200000C68204007EB80000C300026B14604A942
:10621000FEF761F810B1D7F81804A8B1002001AA60
:1062200004994B1C214007EB81010493C96842F893
:106230002010401C0228F3D3019800F0030002282C
:106240000FD001286CD0A0E079680498814203D86F
:106250007868B8600020C6E7204007EB80000C306B
:10626000D5E701984FEA905A01985021B1EB905F21
:1062700001D9554600E05025019865F39F500190E3
:1062800005F10801654800F0EAF9064630007CD0C7
:1062900000F031FA4B46082201A9304600F048FAD6
:1062A00009F1080904992140601A401C80008542C8
:1062B00027D9584C0C34002804D007EB810101F198
:1062C0000C0100E0214601D0024600E02A4602F01F
:1062D000FF0B01D14FF0000402D0A5EB000001E05C
:1062E0004FF00000C5B24B465A46304600F020FA47
:1062F00009EB0B036CB12A462146304600F018FA30
:1063000007E007EB81010C314B462A46304600F08E
:106310000FFA04980AF1030A00EB9A00049034E0A3
:106320000198C0F38310062800D30620019960F37A
:10633000891101910198C0F38310801C81003748B6
:1063400000F08DF9064630001FD000F0D4F94B461E
:10635000082201A9304600F0EBF909F108090025EF
:106360000EE004984B46411C2040049107EB80014D
:106370000C310422304600F0DBF909F104096D1CF0
:106380000198C0F38310A842EBD84EB3D7F810445D
:10639000D7F8180480B1304600F0B3F935E000209A
:1063A000E168497901B1012020B1204631460268F7
:1063B00012689047E0680468002CF0D1304600F085
:1063C000A0F9CDF800806846FBF704FED7F8180462
:1063D00008B90498B8609DF80000FBF71DFE14E0B2
:1063E000D7F8104405E02046016889688847E068CE
:1063F0000468002CF7D10A480A49401AC008022153
:1064000001EB004008A100F019F8FCF78BFE80F0CA
:106410000100E8E66C3900203C2C002068A405004F
:1064200040A40500C0A305004261636B656E647300
:1064300020666C75736865640000000000231A46CE
:1064400002F0C0BB08B5009201236A4602F0BAFB15
:1064500008BD1CB50092019302236A4602F0B2FB0C
:106460001CBD3EB5069C00920193029403236A462C
:1064700002F0A8FB3EBD00002DE9F04707460E469E
:1064800092469846082E3ED898F80C90002088F83E
:106490000C004146504601F061FD0024B44205D293
:1064A0003A5D1AA14046FFF749F903E019A14046B9
:1064B000FFF744F9641C082CF0D317A14046FFF7FE
:1064C0003DF90024B44210D23D5D7E2D06D8F9F787
:1064D000D9FF0068405D10F03E0F00D12E252A46FE
:1064E0000EA14046FFF72AF903E00DA14046FFF751
:1064F00025F9641C082CE5D301224146504601F0E1
:10650000FFFC88F80C90BDE8F087000020253032B1
:1065100078000000202020007C000000256300009F
:106520002000000010B5064901200870054800F061
:10653000E6F8002803D1044800F038F9002010BD27
:106540006C39002068A405007898050002480349CA
:10655000401AC0087047000068A40500C0A30500E9
:1065600013B56846FEF788FA08B100201CBD034841
:10657000009900EBC10000681CBD0000C0A305002D
:1065800070B50848D0F810440125057007E0E068B0
:1065900045712046016849688847E0680468002C16
:1065A000F5D170BD6C3900202DE9FF4707460C9DE1
:1065B0000C46914698462E7B00202873294640467B
:1065C00001F0CCFCB9F1070F41D2DFE809F0040972
:1065D0000F151D27330039462846FFF7AFF836E080
:1065E000394628462268FFF7A9F830E00CCC394636
:1065F0002846FFF7A3F82AE0A06800900CCC3946A3
:106600002846FFF79BF822E0D4E90201CDE900011A
:106610000CCC39462846FFF791F818E0D4E903215D
:10662000A068CDE9012100900CCC39462846FFF73F
:1066300085F80CE0D4E90223D4E90410CDE9021076
:10664000CDE900230CCC39462846FFF777F8002225
:106650002946404601F054FC2E73BDE8FF872DE922
:10666000F04107463D8A2D1F4819C01CB0FBF5F0CC
:1066700000F0FF083846FEF7B7FE044620000AD0B7
:106680000020207101206071E5802646A8F10108F4
:10669000376000250DE00020BDE8F0813846FEF7A8
:1066A000A3FE50B16179491C6171306007600646F4
:1066B0006D1C4545F2D32046EEE7204600F002F877
:1066C0000020E9E72DE9F04101464D790A466B1EAD
:1066D000002001E01268401C9842FBD31768002498
:1066E00005E00E683846FEF7A9FE3146641CAC4250
:1066F000F7D3BDE8F0810121001DFEF74EBEFEF785
:10670000B8BE38B504460121201DFEF767FE009093
:106710009DF80000002802D12046FFF7D3FF38BDC6
:106720001CB501920122009201AAFEF74BF91CBD93
:106730001CB501920022009201AAFEF743F91CBD8C
:1067400010B5064900204870091D0860BFF35F8F2F
:106750000349044800F07AFA002010BD282C0020DC
:1067600010970500C837002008B500200090684643
:10677000FBF730FCF1EE100A20F09F00E1EE100A6A
:10678000BFF35F8F0749402008609DF80000FBF7CA
:1067900043FC00F027FA08B141DF08BD20BF40BF2D
:1067A00020BF08BD84E200E0FBF774BB82680021D3
:1067B000916082681161826851618268D1608268EB
:1067C000516080680160704708B50022425040580F
:1067D000009008BD024A1060101D01607047000063
:1067E0002C760040030103481844C0F81425C0F873
:1067F000101570470070004002494058002800D032
:10680000012070470070004008B503490022084489
:1068100002600068009008BD00700040002804D0AD
:10682000034909680160002070470E20704700008E
:106830000C9905002DE9FE4307460D462846FFF753
:10684000EDFF00287CD100260096019602968DF877
:1068500000704FF001088DF802800620ADF80400AA
:10686000694620202A6869DF3649374A891AC908EB
:10687000012202EB014430B100F058FA02462046F2
:106880003249FFF7DFFD0096019602968DF80180F0
:106890008DF802608DF80360694640202A6869DF40
:1068A00030B100F043FA024620462949FFF7CAFDFD
:1068B0000096019602968DF80070F720ADF8020060
:1068C000694623202A6869DF30B100F02FFA0246BA
:1068D00020462049FFF7B6FD0096019602968DF8F6
:1068E0000080694601202A6869DF30B100F01EFA95
:1068F000024620461849FFF7A5FD019602964FF47F
:10690000B06000906946A1202A6869DF30B100F0CC
:106910000DFA024620461149FFF794FD00960196B4
:1069200002968DF800606946A0202A6869DF30B1C0
:1069300000F0FCF9024620460949FFF783FD0020DC
:10694000BDE8FE8350A40500C0A3050008A1050012
:1069500050A105009CA1050068A00500B4A0050099
:1069600014A005002DE9F0410446D4F8008020462B
:1069700060DF0746164817492268401AC608424594
:1069800014D9022000EB064513A12846FFF756FD57
:10699000284642461CA12368FFF75BFD01F0F0FB8F
:1069A0002168421A284625A1FFF74CFD01245FB15A
:1069B000384600F0BBF9024604EB06402AA1FFF777
:1069C00041FD3846BDE8F0812F480470F9E700002A
:1069D00050A40500C0A30500496E7375666669631F
:1069E00069656E742052414D20616C6C6F636174F7
:1069F000656420666F722074686520536F66744406
:106A000065766963652E00004368616E6765207472
:106A100068652052414D207374617274206C6F63FD
:106A20006174696F6E2066726F6D203078257820F2
:106A3000746F20307825782E000000004D61786951
:106A40006D756D2052414D2073697A6520666F72B5
:106A5000206170706C69636174696F6E2069732066
:106A6000307825782E00000073645F626C655F6586
:106A70006E61626C6528292072657475726E65643A
:106A80002025732E00000000932C002030B5ADF5BA
:106A9000017D15480078002822D04FF4FA7418E0E0
:106AA00005281DD00DF5017DBDE83040FBF7F2B99A
:106AB00004AD0E49684600F0C9F807E002990A687B
:106AC000496828469047684600F0DAF8029800289E
:106AD000F4D1039403A904A861DF0028E8D0DFE71C
:106AE0000DF5017D30BD0000932C002010990500AC
:106AF000F8B5144C2078002817D00120A07001F0C0
:106B00001BFE112813D0022001F02EFE0025009557
:106B10006846FBF75FFA11DF064625709DF8000016
:106B2000FBF77AFA2EB13046F8BD0820F8BD0020F8
:106B3000F8BDA57001F0A2FF032001F015FE0020B2
:106B4000F8BD0000902C00207CB5194D2878002855
:106B500001D008207CBD0120A870002001F0ECFDD0
:106B6000112818D0002001F0FFFD124800680190A4
:106B7000002600966846FBF72DFA0F4901A810DFA2
:106B8000044654B1002028709DF80000FBF744FA39
:106B90002CB120467CBD00207CBD0120F3E7AE7007
:106BA0006E7001F08FFF012001F0DEFD00207CBD42
:106BB000902C0020A4980500151E05000EB508496C
:106BC000684600F043F806E002980168406888478C
:106BD000684600F055F802980028F5D10EBD000077
:106BE000C09805000148007870470000902C0020F4
:106BF00005488178002903D0007818B1FFF778BFE5
:106C000008207047FFF7A0BF902C00201FB503A8F5
:106C10004BDF30B1052815D004B0BDE81040FBF7BC
:106C200039B90949684600F011F807E0029802688E
:106C3000416803989047684600F022F802980028BF
:106C4000E5D0F3E71FBD00002C990500016009683D
:106C50004160AFF3008010B502680CE00021816054
:106C600010BDD1E90034A34203D0416809688160B6
:106C700010BD08314160416853689942F1D1EDE798
:106C8000816800290BD002689268114481604268D3
:106C90005368994203D108324260FFF7DCBF704766
:106CA00070B505460E466C6804E0AA683146904708
:106CB00018B1246820680028F7D120683060266069
:106CC00070BD40680068704741680868002801D0BE
:106CD00002680A60704702460020526806E08B4254
:106CE00003D108681060012070471A461368002B12
:106CF000F5D1704710B50C4A02F594730EE0991A5D
:106D0000C91001EBD171491002EBC1010C6884423A
:106D100001D90B4602E005D201F108029A42EED3F6
:106D2000002010BD486810BD3097050000B5FFF782
:106D3000E1FF002800D1014800BD00001C970500BC
:106D40004FF4A07101EB800080B2704708B50022BB
:106D500042504058009008BD02480068002800D00A
:106D6000012070470004014008480068012110F02C
:106D7000010000D0012028B90448C0227C3880F8E6
:106D80007C23C167012002490860704700E100E0F0
:106D9000180500400246002005490B79002B01D060
:106DA000852070470A6001220A7100224A717047EB
:106DB000982B002010B50220074908604FF482701C
:106DC000FEF770FC05490120086005480168C1F321
:106DD00000410029FAD110BD080300400C0000401A
:106DE00018040040002802D001498001084770477C
:106DF000E19605002DE9F04105460F46284601F0D1
:106E000007F8F0B12846FCF705FA083801F070F8E9
:106E1000032807D0012812D003212846BDE8F041FD
:106E2000FFF7B4B84FF0A04000F5A2600068E8405A
:106E300000F0010008B10321EFE70221EDE7022194
:106E4000EBE7284600F0F0FF002823D02846FCF7A7
:106E5000E1F904464FF4807000EB840082B22046D2
:106E60000D4E06EB8000D0F8101541F00101C0F87E
:106E700010151046FFF7E2F8002F0BD02846FCF75C
:106E8000C9F9064951F82000002803D00120A0408C
:106E9000C6F80403BDE8F08100600040A036002081
:106EA0002DE9FC410C46054611460027DFF8AC8071
:106EB00008EB050090F93000C017401C002801D0F5
:106EC000082747E0A078C0F340022846FCF778F98D
:106ED0000646701C3DD0A078410717D4C0070AD0E1
:106EE0004FF0A04000EB8500D0F8001721F0020120
:106EF000C0F8001707E063782846002100910A4691
:106F00000191FFF729F8284600F074FFA078800768
:106F100016D52178124800EB860000F5A2600268C1
:106F2000104B1A4002604FF4F8524FF4403302EA1B
:106F3000052203EA01410A4301680A43026009E0AD
:106F400008EB0600227810F8481F41EA8211017010
:106F500000E004273846BDE8FC810000A036002090
:106F600000600040FFE0FCFF4FF0A04101F5A2618E
:106F70000968C14001F00100002800D001207047DD
:106F800070B5194D95F85800002801D0082070BD43
:106F90000024661E2046FFF71DF810B1281980F85E
:106FA0003060641CE4B2202CF4D300242046FCF7AB
:106FB000F9F8641CE4B20C2CF8D3002068650B4C83
:106FC0000B49C020087001264FF0E0214020C1F895
:106FD00000014FF4BE70FFF731F8A004C4F80403B9
:106FE00085F85860002070BDA03600200060004089
:106FF00006E400E0034890F85800002800D0012083
:1070000070470000A03600202DE9F8438046042791
:10701000124D00244FF001091BE00020009068464B
:10702000FAF7D8FF09FA04F62E420AD02046FDF7F7
:1070300095F930B90A4841683143416088F8004009
:1070400000279DF80000FAF7E7FF27B1B543641C5D
:10705000E4B2002DE1D13846BDE8F883FFFF01001E
:10706000A82B00202DE9F04107460D461646002DBD
:1070700013D096B100243846FDF7B0F978B1384600
:10708000FDF76CF968B1084800EBC700C0F810556F
:10709000C0F814652046BDE8F0810E20FBE7072408
:1070A000F8E70824F6E7000000F0014070B5054657
:1070B00000242846FDF75EF968B12846FDF78EF9F1
:1070C00018B12846FDF74AF938B105490120A84012
:1070D0000860204670BD0724FBE70824F9E700009C
:1070E00004F501402DE9F04106460D461220264CDC
:1070F000C4F808032549087C022819D00A7C0846F0
:10710000A71590F82E00012A18D00222C4F80423F3
:107110004FF0010881F810804E600D810022CA6096
:1071200038B34D8391F82D103046FFF753FB29E01B
:107130001220C4F804031120BDE8F081CA6822B10E
:107140000220C4F804031120F6E7CE600D8358B97D
:107150003846FFF751FB0028FAD03846FFF754FBBA
:1071600029463046FFF736FB0220C4F8040300200E
:10717000E2E729463046FFF72DFB3846FFF744FB90
:10718000C4F800800020D7E70070004014370020CA
:1071900070B50C46274A117C002901D0112070BD22
:1071A0002179254D09B1012901D10021296002EB86
:1071B00040010B7F1BB912F82D3F5B1C1370E27965
:1071C0000A77227A4A7721786278302301F0030126
:1071D00003EA02121143A2784FF4E06303EA0222A9
:1071E0001143E2784FF4805303EA023211432279CB
:1071F0004FF4E02303EA0242114362794FF4801313
:1072000003EA02521143A2791B0103EA02620B4B0B
:10721000114303EB0012C2F81815227AE179FFF747
:10722000E1FA207908B1012801D10120286000206D
:1072300070BD000014370020007500400070004051
:107240002DE9F0410546204C94F82C00002802D08E
:107250000820BDE8F081103444F8101C28781B4940
:1072600008606878091D0860E878A077012626770D
:107270000020207060776060E0776FF00040144F6E
:10728000C7F808034FF48270FFF7BEFA3002FFF729
:10729000BBFA4FF48A70FFF7B7FAA8780D4940019E
:1072A00008704FF0E0208021C0F800110220C7F8DC
:1072B0000403A07F10B10120C7F804030348F0388D
:1072C00006600020C5E7000014370020F07500407C
:1072D0000070004007E400E0054890F82E00002808
:1072E00001D0002000E0042002490844704700005B
:1072F00014370020007000402DE9F04104460E468E
:1073000017464FF48035B540002B0AD03046FFF7C2
:1073100017FD01462068FFF719FD2068C0F80453E7
:1073200002E02068C0F80853206800EB8600C0F82F
:107330004075BDE8F0810000016801220A60007913
:10734000034A00EB400002EB80000221017270470B
:10735000FC360020F0B4049E4FF480758D40012768
:107360008F4004683D43D4F80072AF43C4F8007204
:107370000468D4F800521D43C4F800523346F0BCF0
:10738000FFF7BABF2DE9F04104460E4620792D499A
:1073900000EB400001EB8007387A002802D008207B
:1073A000BDE8F0813A6070687860002508E0284602
:1073B000FFF7C6FC01462068FFF7C8FC6D1CEDB264
:1073C0006079A842F3D8206840F30730F1780028AC
:1073D00005DB00F1E020490180F8001406E000F030
:1073E0000F0000F1E020490180F8141D206840F3EF
:1073F00007300122002809DB00F01F0102FA01F129
:107400004009800000F1E020C0F800117178206888
:10741000D0F8043561F30103C0F80435B178206871
:10742000D0F8083561F30103C0F8083531782068D9
:10743000D0F8103561F30303C0F810353A7200201C
:10744000AEE70000FC360020044A034902EB80004E
:10745000C0F80016704700003546526E000001402B
:1074600010B504462078002811D109480949A28A9C
:10747000401AC008042101EB004007A1FEF7E2FF1B
:10748000B4F914102069BDE81040F9F767B910BDD0
:1074900040A40500C0A30500415050205220646163
:1074A00074612020424C45202564200033B5C1B0D2
:1074B000002101ABBDF8082102E0445C5C54491C8A
:1074C0009142FAD30B4D0B4842AA6B8801A90C30AC
:1074D000FBF716FA0446082C07D0132C05D0052C10
:1074E00003D0204608B1FAF7D5FC132CEBD043B0FB
:1074F00030BD0000E02A00200149086000F002B819
:1075000004E50140024801680029FCD070470000F2
:1075100000E4014010B500280AD0032808D1022059
:10752000FBF7F8FB002803D0BDE81040FAF7B2BC27
:1075300010BD000010B5FCF7A5FD024AC2E9060126
:1075400010BD0000F82B002010B5054C6068002825
:1075500004D0606801F0B8FB0020606010BD00003E
:10756000F82B00200078002807D104483B214088F0
:1075700076DF002801D0FAF78DBC7047E02A0020A2
:1075800070B50546AE883046FCF738FE0446002C40
:1075900010D04FF6FF7340F2F31205F1080104F129
:1075A0000A00FCF7F5FE607221463046BDE87040E7
:1075B000FBF7E6BF70BD00002DE9F0410546E87B12
:1075C000AE88012829D14FF6FF773846FCF716FE22
:1075D0000446ECB126800020207211480168C4F8EE
:1075E0000A104068C4F80E003B4640F2F31205F161
:1075F000100104F10A00FCF7CBFE60720948C08953
:1076000000280AD121463046BDE8F041FBF7B8BF5B
:10761000BDE8F041042001F0BDB8BDE8F0810000F4
:10762000902B0020F4350020F0B58BB004460D46B9
:1076300000260196A98801AA6069FAF7A1FD0396C0
:1076400002A804900227ADF80C70ADF80E602189F5
:10765000A88803AAADDF002819D1A069002816D098
:107660000498FBF708FA002811D0019E0EB1012002
:107670003070182105A8F8F722FF8DF814700694D1
:10768000A888ADF81C000896A16905A888470BB02A
:10769000F0BDCA7B012A02D18988A0F82414704762
:1076A0002DE9F0418E8800EBC604A41D0279A27179
:1076B000C97B012902D0022905D102E0008820807F
:1076C00001E0408820802288608882421AD91748C9
:1076D00017493346401AC508042000EB0540804690
:1076E00014A1FEF7B6FE21883046A5DF012790B130
:1076F000112812D0FFF71AFB024607EB05401DA127
:10770000FEF7A0FEA179E07981420DD93046BDE8AF
:10771000F041FBF777BF6771F4E7277140463246C7
:107720002149FEF78FFEEDE7BDE8F081C0A305001B
:10773000C0A3050052657175657374696E67207426
:107740006F2075706461746520415454204D545508
:1077500020746F202575206279746573206F6E2008
:10776000636F6E6E656374696F6E20307825782E56
:107770000000000073645F626C655F67617474632E
:107780005F65786368616E67655F6D74755F72656C
:10779000717565737428292072657475726E6564DD
:1077A0002025732E000000006C9B0500F0B58DB005
:1077B00005462C22091D02A8F8F768FEBDF80860EE
:1077C000BDF80C0005EBC607C2B27A731B481C4912
:1077D0003346401AC108042000EB014419A1204699
:1077E000FEF737FEBDF80E20204622A1FEF72AFE46
:1077F000BDF80C20204624A1FEF724FEBDF812207F
:10780000204626A1FEF71EFEBDF81020204627A127
:10781000FEF718FE286900280DD028484169006944
:10782000CDE90001ADF80260787B8DF804002A698B
:107830006946284690470DB0F0BD0000C0A3050082
:10784000C0A3050044617461206C656E6774682094
:107850007570646174656420746F202575206F6E87
:1078600020636F6E6E656374696F6E2030782530AB
:10787000782E00006D61785F72785F6F6374657455
:10788000733A2025750000006D61785F74785F6F32
:1078900063746574733A2025750000006D61785F2C
:1078A00072785F74696D653A202575006D61785F47
:1078B00074785F74696D653A2025750090960500AF
:1078C00070B50C1D228800EBC20625790A480B49C9
:1078D0002B46401AC008042101EB004008A1FEF726
:1078E000B8FD307BA84200D2054629462088BDE875
:1078F0007040FBF787BE0000C0A30500C0A30500D1
:1079000050656572206F6E20636F6E6E656374697B
:107910006F6E203078257820726571756573746597
:107920006420612064617461206C656E67746820F6
:107930006F662025752062797465732E0000000043
:1079400010B58088FCF75AFC0446002C08D060680B
:10795000FAF71EFB08B100F01DFF4FF6FF70208004
:1079600010BD10B50446002084F82E048888B4F8B1
:10797000241488420ED1207900280BD10121204601
:10798000FAF774FD002805D0A16B002902D0BDE8EC
:107990001040084710BD898800EBC100801DFCF72E
:1079A00017BE00002DE9FC4707468D88CE8807EBFF
:1079B000C504A41D204821493346401A4FEAD00887
:1079C000042000EB084081462A461DA1FEF741FD38
:1079D000172E00D217262088B04200D806466680AF
:1079E00000202071009523886288484623A1FEF775
:1079F00038FD21882846B5DF40B1FFF797F90246E8
:107A0000012000EB08402DA1FEF71CFD6079002845
:107A100010D1386900280DD03448C1688068CDE99C
:107A20000001ADF802506088ADF804003A6969467B
:107A300038469047BDE8FC87C0A30500C0A30500F9
:107A400050656572206F6E20636F6E6E656374693A
:107A50006F6E203078257820726571756573746556
:107A60006420616E20415454204D5455206F66208F
:107A700025752062797465732E000000557064616D
:107A800074696E6720415454204D545520746F2002
:107A90002575206279746573202864657369726541
:107AA000643A20257529206F6E20636F6E6E6563C2
:107AB00074696F6E20307825782E000073645F62E1
:107AC0006C655F67617474735F65786368616E6726
:107AD000655F6D74755F7265706C792829207265B9
:107AE0007475726E65642025732E000090960500F3
:107AF0007CB505468E884A8905EBC604A41D2088FE
:107B0000904200D802466280172A00D21722628073
:107B10000F4810493346401AC008042101EB0040C9
:107B20000DA1FEF796FC286970B1607960B1194823
:107B300003C8CDE90001ADF802606088ADF804002B
:107B40002A696946284690470020607120717CBDF3
:107B5000C0A30500C0A30500415454204D54552036
:107B60007570646174656420746F20257520627976
:107B7000746573206F6E20636F6E6E656374696FDA
:107B80006E20307825782028726573706F6E73656B
:107B9000292E00009096050070B588B004460E4668
:107BA00001AAB1886069FAF7EBFA002815D1019DA6
:107BB0002878002811D0A06900280ED0182102A82A
:107BC000F8F77DFC01208DF808000394B088ADF82B
:107BD00010000595A16902A8884708B070BD000093
:107BE0000549C868401CC860082803D90020C8603F
:107BF0000120704700207047B040002010B5104AA7
:107C00000021D1600179002902D0012916D10DE0AF
:107C1000D0E90523D11A4FF48054A14200D3214664
:107C200019448161914209D1012010BD0169491CAB
:107C300001614069814201D1012010BD002010BDC9
:107C4000B040002005484FF08072D0E904138A1834
:107C500043F10001C0E9042170470000F82B002027
:107C60001FB5044608886288904222D18A1C107889
:107C700002281ED1107A042803D0062801D0052836
:107C800017D10020009001900290039002238DF8FC
:107C900000304FF4C073ADF80430127A052A01D1D8
:107CA000ADF8040008886946B0DF002801D061689B
:107CB00088471FBD10B504460888262813D1087AC6
:107CC000012801D002280ED1A078F9F7DDFF014686
:107CD0002046FAF7CBFB002805D0A16B002902D083
:107CE000BDE81040084710BD70470A79012A07D146
:107CF00009884288914203D10121017201F096B9AD
:107D00007047000070B5841D114A2188D2899142C4
:107D10001DD1618902291AD186883046FCF76EFA96
:107D20000546002D13D004F10C00FAF7A4FE28B18B
:107D300029463046BDE87040FBF722BC6868FAF778
:107D400027F9002803D0BDE8704000F023BD70BDC6
:107D5000F4350020F0B587B004460D46AE1DA98865
:107D60006A466069FAF70CFA182101A8F8F7A7FB30
:107D70000294A888ADF80C00009A049231882389F7
:107D8000002705F11200994202D17389022B10D00D
:107D9000A28991420BD1A169002908D08DF8047005
:107DA00005907089ADF81800A16901A8884707B04F
:107DB000F0BD002AFBD0FAF75EFE30B10099012039
:107DC000087002208DF8040004E00098077003207A
:107DD0008DF80400A1690029E9D001A88847E6E7E9
:107DE0000068012803D0022801D00020704701203C
:107DF0007047000010B50549C20800F007008B5C11
:107E00000124844023438B5410BD0000F43600202D
:107E10000449084490F93000082801DB012070472C
:107E200000207047A03600200449084490F9300033
:107E3000082801D20120704700207047A03600209A
:107E40002DE9F0478246DFF890804FF0A0490024EA
:107E500008EB040090F95000401C32D0204600F09E
:107E60003DF8074651463846FDF71CFB48B320460F
:107E700000F03EF8054609EB8700D0F80007C0F394
:107E80000146022E12D002213846FEF77FF801206B
:107E9000B840C9F820053846FBF7BCF958F820204F
:107EA0007AB1032D0AD0022E02D003E00321EBE7C2
:107EB000012D03D0032E04D1022D02D129463846CC
:107EC0009047641C042CC3D35046FCF794FA002856
:107ED000BDD1BDE8F0870000A0360020034908446A
:107EE00090F8500020F0C00070470000A03600203D
:107EF0000249084490F8500080097047A0360020DD
:107F000010B50C46037A052B0CD0407A28B10A48EC
:107F10000AA102682046FDF711FC09A12046FDF7E1
:107F20000DFC04E01AB106A12046FDF707FC20462F
:107F3000BDE81040FDF70FBC6C2C0020257300003D
:107F40000D0A000041DF704710B5FEF7F9FB00286D
:107F500003D0BDE81040F9F79DBF10BD38B5044609
:107F60000D46E388002B06D015A0009016A218A19C
:107F70002846FDF7E3FB217A052920D0607A48B135
:107F8000A088FEF703F9184951F8202017A12846C8
:107F9000FDF7D4FB2846216800F052FFA08800219D
:107FA000FEF7DEFA03461049207A143951F82020F2
:107FB00001B02846BDE830400DA1FDF7BFBB38BD7C
:107FC0001B5B306D000000001B5B313B33316D00EB
:107FD00025734C6F67732064726F7070656420281E
:107FE00025642925730D0A006C2C002025730000E0
:107FF0003C25733E2025733A2000000070B50546ED
:108000000E480F49401AC108032000EB01440DA19E
:108010002046FEF713FA686812A102682046FEF7B0
:1080200011FA686815A142682046FEF70BFA20464F
:10803000BDE8704017A1FEF701BA000040A405009A
:10804000C0A305003D3D3D3D3D3D3D3D7C20666C72
:1080500061736820696E666F207C3D3D3D3D3D3D0E
:108060003D3D0000657261736520756E69743A204C
:1080700009256420627974657300000070726F676F
:1080800072616D20756E69743A20092564206279E9
:10809000746573003D3D3D3D3D3D3D3D3D3D3D3DB8
:1080A0003D3D3D3D3D3D3D3D3D3D3D3D3D3D3D3D00
:1080B0003D3D0000034802490068FDF721B900007A
:1080C000982C00209899050010B5074805490068CC
:1080D000FDF721F90349091F0860002800D001209D
:1080E00010BD0000982C00209899050070B5194C1F
:1080F0000025207A002802D1FFF7E6FFA8B1022070
:108100002072154E3068017989B1012912D00320FF
:1081100098B111281AD003213068FBF7A3FC25720F
:108120006560BDE87040FFF7C5BF656070BD01F0D8
:108130004BF8EDE7FBF76AFCEAE7207C0028F5D175
:10814000BDE8704000210220FDF7BEBD0120207275
:1081500070BD0000B0400020942C002010B5074CEA
:10816000201DFDF717F9002806D1607C002803D1F7
:10817000BDE81040FFF7BABF10BD0000B0400020BE
:1081800002480068800200F1005070470C010010A6
:1081900010B510461A46F8F779F9002010BD10B551
:1081A0004278002140F6B833012A0DD0B0F90420FE
:1081B0009A4201DA521C8280B0F90420032A2BDD96
:1081C0008378012B29D033E0B0F906209A4201DAF6
:1081D000521CC280B0F90620032A1DDB83780124DB
:1081E00043B9037A13B1022B02D003E0047201E019
:1081F000032303721E2A0DDD027A012A02D0032A0C
:1082000003D004E00A22027201E014220272027A10
:10821000427201728180847010BD037A012B02D0FA
:10822000032B03D004E00223037201E00423037252
:108230000F2A02D1037A437201723C2A02D1427A98
:1082400082724172C180817010BD000010B5044679
:10825000142C01D3002010BD21460548FDF78AF8F3
:1082600003482146001FFDF785F8012010BD0000DE
:108270001836002070B506460024054D314605EB42
:108280008400001DFDF760F8641C1E2CF6D370BD41
:108290001036002030B597B00F488168C943169159
:1082A000416816A8FDF77FF816996846FBF7D4F8E1
:1082B0002C2269460BA8F8F7E9F800240BAD05E07D
:1082C00005EB44008088FFF7D5FF641C0B98A042A3
:1082D000F6D817B030BD0000103600200146014826
:1082E000FDF732B81836002070B50020FAF7E6FC2A
:1082F0000C490124002508B14C7000E04D700120AC
:10830000FAF7DCFC07490C3108B14C7000E04D7005
:108310000220FAF7D3FC0349183108B14C7070BD44
:108320004D7070BD004300200846704710B50446EC
:108330002046FBF7C2FA08B1FFF784FC0021204673
:10834000FBF714FA10B12046FFF7FEF80121204692
:10835000FBF70CFA10B12046FFF7ECF8204600F0CE
:1083600003FD2046BDE8104000F03CB82DE9F04781
:1083700007460E464FF00D094FF0000886F80080C2
:10838000D7E90245FBF77EFE221A65EB01030021C7
:108390000846891A984114DAB2F5350F03D3F9F774
:1083A00085FD0E49441822464FF4960300210C48DF
:1083B000FBF78FFA81465FEA090006D10120BDE88C
:1083C000F08700210648FBF7CBF9B9F10D0F03D177
:1083D000384600F079FC30700020F0E7FFFFB40071
:1083E000002C0020F8B50646244D39E0002000247A
:1083F00098B3D0E90212C84370EA020020D068683E
:1084000008B36868D0E90230C91A82410BD201244E
:108410006868D0E90210C94371EA000103D06968B5
:108420001748FEF73DFC002C16D000F087FB0446F1
:1084300069462046FFF79AFF80B1686828B107E0D7
:1084400000F07CFB0CE00124EDE73046FBF739FA45
:108450006C609DF8000018B9F8BD07E00020686066
:108460000748FEF72EFC0028C1D1BFE76868002846
:10847000F2D13046BDE8F840FBF727BAF82B0020D0
:10848000CC96050070B504462078002824D104213C
:108490006068FEF727FE08B1F9F7FCFC6068B0F9E8
:1084A0000620B0F90410A2F50072A1F50071104683
:1084B000F9F7F4FD094D28606168B1F90000B1F9E0
:1084C0000210A0F50070A1F50071F9F7E7FD6860F2
:1084D000BDE87040FCF756BB70BD0000082F0020BF
:1084E00010B50A490020087000F028F800F0AEF836
:1084F00000F090F806480749401AC008032101EB34
:10850000004005A1FDF79AFF10BD0000B034002027
:1085100040A40500C0A30500534141444320484105
:108520004C2073696D706C65206578616D706C6549
:1085300020737461727465642E00000030B58DB0D4
:10854000314841680C9101218DF83010D0E90724A1
:108550008369CDE90A24099302228DF826208DF83B
:108560002710D0E90A45436ACDE9074506938DF8FF
:108570001A208DF81B10D0E90D45036BCDE9044599
:1085800003938DF80E208DF80F10D0E90F34406C56
:10859000CDE9003402908DF802208DF803100CA86C
:1085A0001A49FEF74DFE08B1F9F774FC09A900203D
:1085B000FEF7EEFD08B1F9F76DFC06A90120FEF704
:1085C000E7FD08B1F9F766FC03A90220FEF7E0FD1C
:1085D00008B1F9F75FFC69460320FEF7D9FD08B141
:1085E000F9F758FC04210A48FEF77CFD08B1F9F7B9
:1085F00051FC074804210A30FEF774FD002801D021
:10860000F9F748FC0DB030BD1C92050085840500CB
:108610009C34002008B50A480078FEF747FD08B1F1
:10862000F9F738FC6846FEF7EFFC064A06499DF864
:108630000000FEF717FD9DF80000FEF737FD08BDAE
:108640000C2B002000700040047100403EB5FDF787
:1086500069F808B1F9F71EFC1E4841690069CDE9C7
:10866000010109208DF804001A481B4A01A90830AD
:10867000FEF788FE08B1F9F70DFC164C08342068A7
:10868000D0F81005C2B24BF680300021F7F7EAFEB1
:10869000024600200146009001232046FEF75AFEC4
:1086A0002046FEF749FE246804F5A074FEF714FE88
:1086B00005460A48FEF7A8FC08B1F9F7EBFB0748A6
:1086C0002A4621460078FEF7CDFC002801D0F9F7B4
:1086D000E1FB3EBD1C920500658D05000C2B0020C2
:1086E00038B500210125002809D001280ED0032823
:1086F0000BD1FEF739FBBDE83840FCF7FDBF0C4855
:108700000560BFF34F8FBFF36F8F38BD0091684690
:10871000F9F760FC074C207808B9FCF7CBFFE0685C
:10872000401CE060A5709DF80000F9F775FC38BDAD
:1087300080E100E08C3600203EB5044609496846D9
:10874000FEF784FA08E002990A68496820469047D3
:1087500030B16846FEF794FA02980028F3D13EBD86
:1087600011203EBDA89805003EB50446084968465C
:10877000FEF76CFA07E002990A68496820469047BC
:108780006846FEF77DFA02980028F4D13EBD00004D
:10879000B498050002498969002900D0084770474C
:1087A000F435002010B575DF0446002C04D0112CE0
:1087B00002D02046FFF7EEFF0CB1002010BD0120D3
:1087C00010BD00002DE9F05F8A461546002D22D02D
:1087D00000260327DFF84C900AEB06012A4600200A
:1087E000F8F73AFC06442D1A80B999F800000028E1
:1087F00011D00124DFF830804FF47A4B08F10101E9
:1088000058468847641EF9D17F1E37B1012089F888
:108810000000002DE0D1BDE8F09F002089F80000A5
:10882000F9E70000302C0020709805002DE9F04198
:1088300080460F461446D8F82800002801D00026AC
:1088400032E00720BDE8F081D8F8280006EB4601A9
:1088500000EB8105A988891CFE2901D90C20F1E7CC
:108860002088491C39542088401C80B22080162161
:1088700039542088401C80B22080C119288800F01B
:1088800029FB2188084482B22280A88850B1A968B7
:1088900081B1D31902461846F7F7F8FD2088A98858
:1088A00008442080761CF6B298F82C00B042CBD851
:1088B0000020C7E70720C5E71CB50A4800906946B5
:1088C0000948FCF79FFE08B1F9F7E4FA0748019060
:1088D00001A90748FAF748F8002801D0F9F7DAFAB1
:1088E0001CBD0000A96705005C3000206174050014
:1088F000EC2A0020022280F8312090F82420002A5F
:1089000002D007220A7001E003220A70028A8A81DB
:108910000022C0F8202400F226424A60C068886025
:1089200000207047012280F831200022C0F8202466
:1089300000F2264048608A6002200870802088810A
:108940000020704770B504460D466069A860208B12
:10895000A88194F82400002803D0062084F83C0065
:1089600002E0012084F83C00204600F051FB58B1A1
:108970000220287504212046FBF750F900280BD16E
:10898000052084F8310002E0032084F8310004F56A
:108990008260C4F82004002070BD70B504460D4606
:1089A000E069A860208CA88194F82400062600289D
:1089B00002D084F83C6002E0012084F83C002046AC
:1089C00000F026FB50B10220287504212046FBF759
:1089D00025F900280AD184F8316002E0042084F8E7
:1089E000310004F58260C4F82004002070BD0A78CC
:1089F00022F00F0222F0F0020A70062809D2DFE806
:108A000000F003091119212922F00F0020F0F000D5
:108A10000870704722F00F00401C20F0F00010306A
:108A20000870704722F00F00401C20F0F00020304A
:108A30000870704722F00F00401C20F0F00030302A
:108A40000870704722F00F00801C20F0F0001030FA
:108A50000870704722F00F00801C20F0F0002030DA
:108A600008707047002805D1034901204870002094
:108A7000FAF7ACBC704700008C36002010B5162009
:108A8000F8F7F8FE48B10D4882684FF480013AB11A
:108A9000016821F48001016008E042F2010006E073
:108AA00007480160BFF34F8FBFF36F8F002000288E
:108AB00003D0BDE81040F9F7EDB910BDBC37002078
:108AC00080E100E010B51620F8F7D4FE98B1124806
:108AD00000784009082811D20121814011F0EC0FE3
:108AE0000CD00E4882684FF4800152B1016841F405
:108AF0008001016007E042F2010005E042F202005D
:108B000002E0074801600020002803D0BDE81040C3
:108B1000F9F7C0B910BD000016E400E0BC37002032
:108B200000E100E010B500F009F8002803D04FF094
:108B3000FF328260C260F6D110BD000010B503485C
:108B4000FEF7C2F80028FFD110BD0000CC9605004A
:108B500010B504460120FAF7B1F810B102202070D8
:108B600010BD0020FAF7AAF810B10B20207010BD3C
:108B70000020207010BD0000054901EB500109786C
:108B8000C00701D00809704701F00F0070470000CE
:108B900044370020C207002A02D04FF00F0201E044
:108BA0004FF0F00201D04FEA0111054B03EB5000EA
:108BB000037803EA020343EA0103037070470000ED
:108BC000443700202DE9F84F82468B4691461F46D8
:108BD0001E480568012269463846FAF737FADFF879
:108BE000708048B3009EB01C002408E00146401C81
:108BF000294008EB810159F82420CA60641CBC425A
:108C0000F4D34FEA1A44FAF7A1FD44EA0041701C7C
:108C1000284008EB8000C1602E4008EB8600C16848
:108C20006AF3C50167F389116BF39F2121F00301FA
:108C3000491C21F00401C16098F80000002803D00D
:108C4000FDF7CAFA0028FBD1BDE8F88F3C2C0020C4
:108C50006C3900202DE9F04107460D4614460026E8
:108C6000D80705D113E06D1C761C3846FAF742FA96
:108C700029780029F7D104E0641E20213846FAF74C
:108C800039FAB44201D9002CF6D1BDE8F0814DB1DA
:108C90002846F7F73BFC064604E0641E20213846D0
:108CA000FAF728FAB44206D9002CF6D103E06D1C7D
:108CB0003846FAF71FFA29780029F8D1E5E7401A73
:108CC00020F07F4070470000F8B504460025234897
:108CD000007800283FD0A4B3FBF7D4F9D4E90223ED
:108CE000801A99412ED3002600966846F9F772F94A
:108CF000206910B9691EA160E1609DF80000F9F7D4
:108D00008BF9D4E90510884700966846F9F762F9AF
:108D100022695AB1D4E90201C34373EA010305D0C1
:108D200080187141C4E90201012600E000269DF887
:108D30000000F9F771F926B121460948FDF7B0FFA7
:108D4000012508E0D04370EA030004D0214604481E
:108D5000FDF7A6FF01252846F8BD0000F82B0020EE
:108D6000CC9605007047000038B51A4C694620685B
:108D7000FCF7D1FA184D2AE0017821B101290ED073
:108D800002291CD117E04168D1E90202C04370EA10
:108D9000020014D00F480830FDF782FF0FE0416851
:108DA0006868814202D10020686008E00948083004
:108DB000FDF791FF03E0FFF7B5FE0120287069463B
:108DC0002068FCF79DFA69462068FCF7A4FA0028A1
:108DD000D2D138BDC4960500F82B0020F8B5044662
:108DE0000D460A4E69463068FCF77CFA58B10470AB
:108DF000456069463068FCF79CFA10B10448FAF700
:108E000049FD0020F8BD0420F8BD0000C49605000F
:108E1000002C002003488068410803480022406875
:108E2000F9F78EB8C02B0020BC96050010B5F9F7F5
:108E300057F8002803D0BDE81040F9F72BB810BD53
:108E40007047FEB506460F4614460025009501956D
:108E5000029539466846F7F760FB3846F7F756FB48
:108E60003D2269460DF80020084445703046F7F76A
:108E700031FB10B90120FEBD401C01783D29FBD11A
:108E800000E0401C01783D29FBD002E004F8011B02
:108E9000401C0178262901D00029F7D12570002037
:108EA000FEBD30B51488E51C9D4201D90C2030BDB3
:108EB00002230B5513885B1C9BB213800A24CC54ED
:108EC00013885B1C9BB21380C8541088401C108010
:108ED000002030BD0870000A487002207047000072
:108EE00010B514210448F7F7EAFA04480068FCF7C3
:108EF000DDF9002010BD0000B04000209899050069
:108F00002DE9F05F8346DDE90A4A8846174699460F
:108F10004046012602E0B0FBF7F0761CB842FAD2D8
:108F2000B14500D94E465FEACA7012D18CB15FEAF2
:108F30008A7002D5B9F1000F01D0202506E0302556
:108F400004E0641E29465846FAF7D4F80CB1A6424C
:108F5000F7D30125B9F1010F02D9A9F1010918E0F0
:108F6000B8FBF5F0B84214D2DFF84090B8FBF5F04A
:108F700000FB158819F800105846FAF7BBF8B5FB46
:108F8000F7F5002DF2D15FEACA7000D044B9BDE810
:108F9000F09F7D43DEE7641E20215846FAF7AAF8C9
:108FA000002CF4D0A642F6D3F1E70000E6960500C7
:108FB000F8B50546A8B2FBF721F90446002C0ED0FF
:108FC000124F207A397B88420AD2A8B204F10A01F2
:108FD000FFF7E8FB002802D0207A401C2072F8BD81
:108FE00000262672387C38B1A8B23B2176DF18B152
:108FF000082801D0FFF7CEFB79690029EFD08DF862
:109000000060ADF8025068468847F8BDF43500208E
:1090100010B54179002907D090F82E1421B900F03D
:10902000A4F808B1012010BD002010BD30B40446E2
:10903000207A00280AD06088002166DF20B111283C
:1090400006D0616830BC08470020207230BC7047F1
:1090500001202072FAE770B504460D462046FAF763
:109060006DF8002807D04268002A04D0294620461F
:10907000BDE87040104770BD2DE9FC410746DDE9B1
:10908000084516469846434602223846CDE9004533
:1090900000F00EF8002809D1434610223146384628
:1090A000CDE9004500F004F80028FFD1BDE8FC81BF
:1090B0002DE9FC5F8046DDE90C4E8A4693461F464B
:1090C0000026B4F80090002532E0D8F8040000EB48
:1090D000850000680090002201A9684664DF00282E
:1090E0000DD19DF80410594521D10EB1002200E0A8
:1090F0000222208811440144714502D90C20BDE8A8
:10910000FC9F46B9401C80B2208007F800A0208850
:10911000401C20800126208801A9C219684664DF0E
:109120000028ECD120889DF80410084420806D1C94
:10913000B8F80000A842C8DC56B12088A0EB0900AE
:10914000401E80B2FF2801D90C20D8E707F809009B
:109150000020D4E710B5044601E0FEF7F3FE2046F8
:10916000FCF7B8FC0028F8D110BD90F83004704727
:10917000002070472DE9F84F0646DDF828A00F467D
:10918000904699460F4D69462868FCF7ABF80446AF
:10919000B4B11C212046F7F792F900202071266017
:1091A000C4F808A02761C4F80C80C4F8149069467C
:1091B0002868FCF7BEF8FEF7D1FF0020BDE8F88F65
:1091C0000420FBE798990500D0E90521521A4FF4D5
:1091D00080539A4200D31A460123B3EB920F01D277
:1091E000920800E0012203690B44C068014418465C
:1091F00029DF704701000000D007000006000000D2
:1092000001000000D007000006000000341200003A
:109210003412000034120000341200000100060075
:109220000100060000A00140010600000000000649
:10923000000000000000000002000001000000002B
:10924000000000000200000200000000000000001A
:109250000200000300000000000000000200000403
:1092600000000000000000000100000001000000FC
:1092700002000000020000000300000004000000E3
:1092800004000000050000000600000006000000C9
:1092900007000000070000000800000009000000AF
:1092A000090000000A0000000B0000000B00000095
:1092B0000C0000000C0000000D0000000E0000007B
:1092C0000E0000000F000000100000001000000061
:1092D0001100000011000000120000001300000047
:1092E000130000001400000014000000150000002E
:1092F0001600000016000000170000001800000013
:109300001800000019000000190000001A000000F9
:109310001B0000001B0000001C0000001C000000DF
:109320001D0000001E0000001E0000001F000000C5
:109330001F000000200000002100000021000000AC
:109340002200000022000000230000002400000092
:109350002400000025000000250000002600000079
:10936000270000002700000028000000280000005F
:1093700029000000290000002A0000002B00000046
:109380002B0000002C0000002C0000002D0000002D
:109390002E0000002E0000002F0000002F00000013
:1093A00030000000300000003100000032000000FA
:1093B00032000000330000003300000034000000E1
:1093C00034000000350000003500000036000000C9
:1093D00037000000370000003800000038000000AF
:1093E00039000000390000003A0000003A00000097
:1093F0003B0000003B0000003C0000003D0000007E
:109400003D0000003E0000003E0000003F00000064
:109410003F0000004000000040000000410000004C
:109420004100000042000000420000004300000034
:10943000430000004400000044000000450000001C
:109440004500000046000000470000004700000003
:1094500048000000480000004900000049000000EA
:109460004A0000004A0000004B0000004B000000D2
:109470004C0000004C0000004D0000004D000000BA
:109480004D0000004E0000004E0000004F000000A4
:109490004F0000005000000050000000510000008C
:1094A0005100000052000000520000005300000074
:1094B000530000005400000054000000550000005C
:1094C0005500000056000000560000005600000045
:1094D000570000005700000058000000580000002E
:1094E00059000000590000005A0000005A00000016
:1094F0005B0000005B0000005B0000005C000000FF
:109500005C0000005D0000005D0000005E000000E7
:109510005E0000005E0000005F0000005F000000D1
:1095200060000000600000006100000061000000B9
:1095300061000000620000006200000063000000A3
:10954000630000006300000064000000640000008D
:109550006500000065000000660000006600000075
:10956000660000006700000067000000680000005F
:109570006800000068000000690000006900000049
:10958000690000006A0000006A0000006B00000033
:109590006B0000006B0000006C0000006C0000001D
:1095A0006D0000006D0000006D0000006E00000006
:1095B0006E0000006E0000006F0000006F000000F1
:1095C0006F000000700000007000000071000000DB
:1095D00071000000710000007200000072000000C5
:1095E00072000000730000007300000073000000B0
:1095F000740000007400000074000000750000009A
:109600007500000075000000760000007600000084
:10961000770000007700000077000000780000006D
:109620007800000078000000790000007900000058
:1096300079000000790000007A0000007A00000044
:109640007A0000007B0000007B0000007B0000002F
:109650007C0000007C0000007C0000007D00000019
:109660007D0000000607161B1C191A00282B00207D
:10967000482B0020682B0020060003001D2C05004D
:10968000070003001D2C0500160003001D2C05001B
:10969000770A000000000000770A000000000000C8
:1096A0007ADA0000000000009ECADC240EE5A9E082
:1096B00093F3A3B50000406E0000005003000000CB
:1096C000D82B0020543700200100060000000000C5
:1096D000182C00201D3405000000000000000000D0
:1096E0000338FDD8704730313233343536373839A6
:1096F00041424344454600000000000000000000D5
:109700000000000000000000000000000000000059
:10971000F89605001097050004000000556E6B6E6A
:109720006F776E206572726F7220636F64650000E0
:1097300000000000389F050001000000E49D0500C6
:1097400002000000D89B050003000000589E0500A1
:1097500004000000AC9E0500050000008C9D050083
:1097600006000000289D050007000000949E0500EB
:1097700008000000A09D050009000000049E0500EF
:109780000A000000209F05000B000000C09B0500A0
:109790000C000000B89D05000D000000889F05002A
:1097A0000E000000849E05000F000000C09E050012
:1097B00010000000F49E0500110000009C9F0500B1
:1097C00012000000709F0500130000000C9F0500B0
:1097D00080000000409D0500810000007C9C050089
:1097E000820000003C9C0500830000001C9C0500DA
:1097F00084000000589C050085000000649D050061
:10980000860000006C9E050090000000089D050089
:1098100091000000FC9B050092000000CC9D05001B
:1098200000820000D49E050001820000209E0500F9
:10983000028200003C9E050000840000989C050008
:1098400001840000449F050002840000E09C0500A4
:1098500003840000BC9C0500A9600500A76005000A
:10986000A1600500000000000000000000000000F2
:109870000338FDD870470000D43800207F00000076
:10988000543900203031323334353637383941429B
:1098900043444546BCA40500C4A4050000000000E4
:1098A000000000000100000794980500A49805003E
:1098B00008000000CC980500DC98050008000000B6
:1098C000DC980500EC98050008000000E4A4050001
:1098D000F4A405000000000000000000D4A405006E
:1098E000E4A4050000000000000000007CA40500C6
:1098F00084A4050084A40500A4A40500A4A4050074
:10990000B4A40500B4A40500BCA40500D82A002016
:10991000EC9805000C99050008000000C4A405009F
:10992000D4A4050000000000000000001C99050000
:109930002C990500080000006E72665F6673746FF4
:10994000726167655F696E6974006E72665F6673E7
:10995000746F726167655F756E696E6974006E72AF
:10996000665F6673746F726167655F7265616400DC
:109970006E72665F6673746F726167655F77726936
:109980007465006E72665F6673746F726167655F9F
:109990006572617365000000144000200010000033
:1099A0000400000001000000C9410500E18E05002F
:1099B0009181050075910500BD39050029830500D9
:1099C0007191050081430500D02E002065726173FE
:1099D000655F666C6173685F6164647200000000BB
:1099E0006E000000000000000A00000018FCFFFFED
:1099F000E8030000030201000040404040404040B6
:109A00004040414141414140404040404040404051
:109A100040404040404040404005020202020202F5
:109A20000202020202020202022020202020202044
:109A30002020200202020202020290909090909058
:109A40001010101010101010101010101010101016
:109A5000101010100202020202028888888888888A
:109A60000808080808080808080808080808080876
:109A7000080808080202020240000000F9990500E7
:109A800052657175657374696E6720746F207570A7
:109A90006461746520415454204D545520746F20E6
:109AA0002575206279746573206F6E20636F6E6E0A
:109AB000656374696F6E203078257820287265742C
:109AC0007279292E0000000073645F626C655F6725
:109AD00061705F646174615F6C656E6774685F7507
:109AE00070646174652829202872657175657374C6
:109AF00029206F6E20636F6E6E656374696F6E20D0
:109B0000307825782072657475726E6564202573CF
:109B10002E00000054686520726571756573746568
:109B20006420636F6D62696E6174696F6E206F6629
:109B300020545820616E64205258207061636B6518
:109B400074206C656E6774687320697320746F6F1E
:109B5000206C6F6E67206279202575206D696372B5
:109B60006F7365636F6E64732E00000073645F62D1
:109B70006C655F67617474635F65786368616E6765
:109B8000655F6D74755F72657175657374282920E2
:109B90006F6E20636F6E6E656374696F6E203078D0
:109BA00025782072657475726E65642062757379AC
:109BB0002C2077696C6C2072657472792E0000001D
:109BC0004E52465F4552524F525F494E56414C49A4
:109BD000445F4441544100004E52465F4552524F4B
:109BE000525F534F46544445564943455F4E4F5488
:109BF0005F454E41424C4544000000004E52465FD6
:109C00004552524F525F464541545552455F4E4F63
:109C1000545F454E41424C45440000004E52465F61
:109C20004552524F525F4D555445585F554E4C4F1B
:109C3000434B5F4641494C45440000004E52465F4D
:109C40004552524F525F4D555445585F4C4F434B10
:109C50005F4641494C4544004E52465F4552524F83
:109C6000525F4D555445585F434F4E445F494E49EE
:109C7000545F4641494C4544000000004E52465F47
:109C80004552524F525F4D555445585F494E4954C5
:109C90005F4641494C4544004E52465F4552524F43
:109CA000525F424C455F495053505F52585F504B92
:109CB000545F5452554E4341544544004E52465F02
:109CC0004552524F525F424C455F495053505F508E
:109CD0004545525F52454A45435445440000000003
:109CE0004E52465F4552524F525F424C455F49507B
:109CF00053505F4C494E4B5F444953434F4E4E4582
:109D000043544544000000004E52465F4552524FB6
:109D1000525F4150495F4E4F545F494D504C454D45
:109D2000454E5445440000004E52465F4552524F46
:109D3000525F4E4F545F535550504F52544544005C
:109D40004E52465F4552524F525F4D4F44554C451F
:109D50005F4E4F545F494E495449414C495A45441E
:109D6000000000004E52465F4552524F525F4D4F29
:109D700044554C455F414C52454144595F494E4919
:109D80005449414C495A4544000000004E52465F38
:109D90004552524F525F4E4F545F464F554E44000E
:109DA0004E52465F4552524F525F494E56414C49C2
:109DB000445F5354415445004E52465F4552524F02
:109DC000525F444154415F53495A45004E52465FE9
:109DD0004552524F525F494F5F50454E44494E479E
:109DE000000000004E52465F4552524F525F53569C
:109DF000435F48414E444C45525F4D495353494E91
:109E0000470000004E52465F4552524F525F494E46
:109E100056414C49445F4C454E47544800000000B1
:109E20004E52465F4552524F525F4452565F54570E
:109E3000495F4552525F414E41434B004E52465F8F
:109E40004552524F525F4452565F5457495F4552F4
:109E5000525F444E41434B004E52465F4552524F73
:109E6000525F494E5445524E414C00004E52465F9F
:109E70004552524F525F53544F524147455F4655EA
:109E80004C4C00004E52465F4552524F525F4E5569
:109E90004C4C00004E52465F4552524F525F494E65
:109EA00056414C49445F504152414D004E52465F2D
:109EB0004552524F525F4E4F5F4D454D00000000DE
:109EC0004E52465F4552524F525F464F52424944AE
:109ED00044454E004E52465F4552524F525F4452E7
:109EE000565F5457495F4552525F4F56455252553F
:109EF0004E0000004E52465F4552524F525F494E4F
:109F000056414C49445F4144445200004E52465F22
:109F10004552524F525F5245534F5552434553009D
:109F20004E52465F4552524F525F494E56414C4940
:109F3000445F464C414753004E52465F535543439E
:109F4000455353004E52465F4552524F525F424C6A
:109F5000455F495053505F4348414E4E454C5F4129
:109F60004C52454144595F455849535453000000F1
:109F70004E52465F4552524F525F434F4E4E5F43E3
:109F80004F554E54000000004E52465F4552524F0E
:109F9000525F54494D454F55540000004E52465FA4
:109FA0004552524F525F4255535900007761726ECD
:109FB000696E670064656275670000001B5B313B7A
:109FC00033306D001B5B306D000000001B5B313BCC
:109FD00033316D001B5B313B33326D001B5B313B1A
:109FE00033336D001B5B313B33346D001B5B313B06
:109FF00033356D001B5B313B33366D001B5B313BF2
:10A0000033376D00696E666F000000006572726F15
:10A010007200000073645F626C655F6366675F7304
:10A02000657428292072657475726E6564202573C5
:10A03000207768656E20617474656D7074696E67F1
:10A0400020746F2073657420424C455F474154541F
:10A05000535F4346475F534552564943455F434824
:10A06000414E4745442E000073645F626C655F6338
:10A0700066675F73657428292072657475726E65F2
:10A0800064202573207768656E20617474656D7037
:10A0900074696E6720746F2073657420424C455F4D
:10A0A000434F4D4D4F4E5F4346475F56535F5555A7
:10A0B00049442E0073645F626C655F6366675F731B
:10A0C000657428292072657475726E656420257325
:10A0D000207768656E20617474656D7074696E6751
:10A0E00020746F2073657420424C455F474154547F
:10A0F000535F4346475F415454525F5441425F535C
:10A10000495A452E0000000073645F626C655F630E
:10A1100066675F73657428292072657475726E6551
:10A1200064202573207768656E20617474656D7096
:10A1300074696E6720746F2073657420424C455FAC
:10A14000434F4E4E5F4346475F4741502E0000004D
:10A1500073645F626C655F6366675F73657428290B
:10A160002072657475726E6564202573207768654A
:10A170006E20617474656D7074696E6720746F20F1
:10A1800073657420424C455F4741505F4346475FCB
:10A19000524F4C455F434F554E542E0073645F62DF
:10A1A0006C655F6366675F736574282920726574E8
:10A1B00075726E6564202573207768656E20617402
:10A1C00074656D7074696E6720746F207365742098
:10A1D000424C455F434F4E4E5F4346475F474154B5
:10A1E000542E0000616464725F69735F77697468FC
:10A1F000696E5F626F756E647328705F66732C2082
:10A20000706167655F616464722C20286C656E20E4
:10A210002A20705F66732D3E705F666C6173685FA5
:10A22000696E666F2D3E65726173655F756E6974E8
:10A23000292900005B2E2E5C2E2E5C2E2E5C2E2EED
:10A240005C2E2E5C2E2E5C636F6D706F6E656E746F
:10A25000735C696E5F6961705C696E5F6961702EC5
:10A26000635D5B25735D5B4C696E653A2025645DBB
:10A270003A20200A000000006E72665F6673746FF9
:10A28000726167655F69735F627573793D202564EC
:10A2900020666C6173685F646F776E5F6E3D20252A
:10A2A0006420202045524153455F57524954455F31
:10A2B000524553554C545F666C61672020256400FD
:10A2C0006E72665F626C655F6761747400000000A7
:10A2D000626C655F6E757300636C6F636B0000008A
:10A2E000434C4F434B0000004750494F544500003A
:10A2F00050525300554152540000000055415254F1
:10A300004500000054494D4552000000534141446E
:10A310004300000050504900574454006170705F82
:10A32000627574746F6E00006170705F74696D6542
:10A33000720000007077725F6D676D74000000003E
:10A34000736F72746C697374000000007274745FD0
:10A350006C6F675F6261636B656E64006170700053
:10A360006E72665F736468006E72665F7364685FC6
:10A37000626C65006E72665F7364685F736F630022
:10A380006E72665F6673746F7261676500000000CD
:10A39000F4A40500D82A00207C040000060705006C
:10A3A00094A60500542F00208C340000641805008A
:10A3B00058980500000000004CA30500342C002034
:10A3C000C0A2050000000404D0A2050000000000A7
:10A3D000D8A2050000000000E0A205000000000077
:10A3E000E8A2050000000000F0A205000000000047
:10A3F000F4A2050000000000FCA20500000000001F
:10A4000004A30500000000000CA3050000000000EC
:10A4100014A305000000000018A3050000000000C0
:10A420001CA305000000000028A305000000000098
:10A4300034A305000000000040A305000000000058
:10A440005CA305000000040460A3050000000303F2
:10A4500068A305000000030374A3050000000303C4
:10A4600080A3050000000404482C0020402C00209C
:10A47000482C002014380020180000005128050046
:10A4800000000000FD54050048300020472405006E
:10A4900068300020E5270500000000002D28050099
:10A4A00000000000492A0500EC2A00202F56050074
:10A4B0005C300020B926050000000000915C05001A
:10A4C00000000000658A050000000000C95C05006E
:10A4D000000000008D6A0500000000000D6C050002
:10A4E00000000000E186050000000000A95C0500F6
:10A4F0000000000013082B132001320414FFFF1486
:10A50000120102170213D82A022C205AFF01095601
:10A51000200150091F7015100140110A30045859CC
:10A5200004011C140CA00514AC9F051A04081AB4ED
:10A53000081AC4041ABC041ACC041AD4041ADC0481
:10A540001AE4041AEC041AF4041AFC04F99F310505
:10A5500020FE0FDCBA1459534D12302808C1814037
:10A5600001C0804104690C2908E918A91C091A30A6
:10A57000091638093660092E70092F6000FF00C0E7
:10A58000C101C30302C2C60607C705C5C404CC0C7B
:10A590000DCD0FCFCE0E0ACACB0BC90908C8D818EB
:10A5A00019D91BDBDA1A1EDEDF1FDD1D1CDC14D4FB
:10A5B000D515D71716D6D21213D311D1D010F0302B
:10A5C00031F133F3F23236F6F737F53534F43CFC3B
:10A5D000FD3DFF3F3EFEFA3A3BFB39F9F83828E8EB
:10A5E000E929EB2B2AEAEE2E2FEF2DEDEC2CE424BB
:10A5F00025E527E7E62622E2E323E12120E0A0602B
:10A6000061A163A3A26266A6A767A56564A46CACFA
:10A61000AD6DAF6F6EAEAA6A6BAB69A9A86878B86A
:10A62000B979BB7B7ABABE7E7FBF7DBDBC7CB4747A
:10A6300075B577B7B67672B2B373B17170B050902A
:10A6400091519353529296565797559594549C5CBA
:10A650005D9D5F9F9E5E5A9A9B5B9959589888486A
:10A6600049894B8B8A4A4E8E8F4F8D4D4C8C44843A
:10A6700085458747468682424383418180B2405A5E
:10A68000FF010155041090D00324193E051B600200
:04A690007812080034
:0400000500050201EF
:00000001FF
